:1073B900758400852FD28530D3E4F530F52F303828
:1073C90010E50D852EF0A4252FF52FE5F03530F5C4
:1073D90030229073F5303E031273E522E50E251B2A
:1073E900F50EE51F351AF51F93F50D227F82858865
:1073F9008C8F9295989B9EA1A4A7AAADB0B3B6B95C
:10740900BBBEC1C3C6C9CBCED0D3D5D7D9DCDEE08C
:10741900E2E4E6E7E9EBEDEEF0F1F2F4F5F6F7F880
:10742900F9FAFBFCFCFDFDFEFEFEFEFEFEFEFEFE85
:10743900FEFDFDFCFCFBFAFAF9F8F7F6F4F3F2F0BD
:10744900EFEDECEAE8E7E5E3E1DFDDDBD8D6D4D11F
:10745900CFCDCAC8C5C2C0BDBAB7B4B2AFACA9A670
:10746900A3A09D9A9794908D8A8784817E7A777458
:10747900716E6B6865625F5C595653504D4A47445B
:10748900423F3C393734322F2D2A282624211F1D0B
:107499001B1918161412110F0E0C0B0A08070605F2
:1074A90004040302020101000000000000000000C2
:1074B9000001010202030405060708090A0B0D0E63
:1074C9001011131516181A1C1E20222427292B2ED9
:1074D900303335383A3D404245484B4E5154565960
:0C74E9005C606366696C6F7275787B7F75
:107AB800D2F4C2F5C2F675840F85F0C81279327413
:107AC80003127B071279227403127B0712791112B1
:107AD80079117403127B071279117402127B071251
:107AE80079117428127B737406127B73740E127BDF
:107AF800737401127B731279227480127B7322C013
:107B080000A2E092F3A2E192F2A2E292F1A2E39241
:107B1800F0D2F475840F85F0C8C2F47830D8FE85A9
:107B2800F0C87830D8FED00022C00075840FA2E4D7
:107B380092F3A2E592F2A2E692F1A2E792F0D2F4D1
:107B480085F0C8C2F47830D8FE85F0C87830D8FE01
:107B5800D00022EF75840FD2F5C2F685F0C8127BEB
:107B680031127911127B071279112275840FC2F52F
:107B7800C2F685F0C8127B31127911127B0712798F
:107B88001122EF14A2E492E6C2E4D2E7127B732238
:107B9800740F127B7322740D127B73227F01127B88
:107BA8008A78107F20127B5BD8F9227F11127B8A9A
:0A7BB80078107F20127B5BD8F922C1
:10727C00C293758400D2C2C2C6D2C6C2C4D2C5C221
:10728C00C330C3FD74A0F5C2C2C5C2C330C3FD8EEA
:10729C00C2C2C330C3FD8FC2C2C330C3FD8DC2C2D4
:1072AC00C330C3FDD2C4C2C320C4FD127922D29311
:1072BC0022758400C2C3D2C530C3FD74A0F5C2C20E
:1072CC00C5C2C330C3FD8EC2C2C330C3FD8FC2C2A0
:1072DC00C330C3FDC2C4D2C5C2C330C3FD74A1F553
:1072EC00C2C2C5C2C330C3FDC2C2C2C330C3FD8556
:1072FC00C207D2C4C2C320C4FD22D2C2C2C6D2C6E7
:10730C00D2C4C2C320C4FD22C293758400D2C2C2AF
:10731C00C6D2C6C2C4D2C5C2C330C3FD74A0F5C2A6
:10732C00C2C5C2C330C3FD8EC2C2C330C3FD8FC23F
:10733C00C2C330C3FD8C838D827B80E0A3F5C2C2B7
:10734C00C330C3FDDBF5D2C4C2C320C4FD12792205
:10735C00D29322758400C2C3D2C530C3FD74A0F58C
:10736C00C2C2C5C2C330C3FD8EC2C2C330C3FD8FFF
:10737C00C2C2C330C3FDC2C4D2C5C2C330C3FD74C4
:10738C00A1F5C2C2C5C2C330C3FD8C838D82C2C3FA
:10739C0030C3FDE5C2F0A31BBB01F3C2C2C2C330B4
:0D73AC00C3FDE5C2F0D2C4C2C320C4FD225F
:030003000255445F
:01000B0032C2
:0300130002762C46
:10641C0075FF0775FFDE75FFAD75840F75E10775A8
:10642C00E21475E34475840F75A43575A50975A63A
:10643C00BB75A7FF759CFF759D00759EF0759FF849
:10644C0075D8FF75E8FF75F80F75AD0F758401757C
:10645C00893075888F75840275893075888F75843D
:10646C000F758A80758C67780874FF000000000037
:10647C0000000000000000D5E0F1D8EDE58C30E71D
:10648C00FB759701758A0043890475840075B710F4
:10649C0075840F438901758D02758F01758E047497
:1064AC0080D5E0FD438902E58930E4FB75970275E0
:1064BC00840075D10775840075BB0175BA0075BC75
:1064CC00F075C70075C60075C5FF75C4FF75E8008B
:1064DC0075840275BB0475BA0075BCF175C6007580
:1064EC00C4FF75E88075840075D48475840175D4F7
:1064FC0084758400C2F8759A47759D1A75F80175F4
:10650C00870075840075B90075A9007591007598A0
:10651C005075840175989075840075C04075C300E2
:10652C0075CFC9758400758E1075892175880575B0
:10653C008400758A00758BE0758CF4758DE043884A
:10654C004075840075C90075CA0075CB0075CC0008
:10655C0075CD0075840175C91875CA8075CBFB752E
:10656C00CDFB75CC80D2CA75840275C91875CAA6C4
:10657C0075CBAF75CDAF75CCA6D2CA75840075EF4F
:10658C000275A8AC75B83D75E6B075E71D75F600DB
:10659C0075F741789D760A769E780A789F7606750F
:0765AC00A8959000007F009C
:1065B3007E20E4F0A3DFFCDEFA789D760A789E76EF
:0E65C3000A789F7606D29375E8FF12730622BF
:10788B0075840FD2FD2275840FC2FD22E490FC009B
:10789B00732275840FD2EA2275840FC2EA22758493
:1078AB000FA2EC2275840FD2FE2275840FC2FE222A
:1078BB0075840FC2FF2275840FD2FF2275840FA22D
:1078CB00FA2275840FA2F92275840FA2DD22A292EF
:1078DB002275840FA2DA2275840FA2DB2275840F26
:1078EB00A2D82275840FA2D922000000000000004C
:1078FB00000000000000000000000000000000007D
:10790B00000000000022C000C001790878B4D8FE46
:10791B00D9FAD001D00022C000C0E078997605E6F4
:10792B0070FDD0E0D00022C000C0E07899760FE661
:10793B0070FDD0E0D00022EF75F06484243090000D
:10794B005CF0E5F0A375F00A842430F0A3E5F02495
:10795B0030F022EF75F06484243090005CF0E5F099
:10796B00A375F00A842430F0A3E5F02430F09000E6
:09797B005CE0B4300B7420F0A3B1
:10798400E0B430037420F02275F06484F6E5F00866
:1079940075F00A84F608A6F00822850607222285D7
:0379A400050622B3
:10554400758400C2CA85CC3985CD3875CC0075CD3B
:1055540000D2CA10CF02D25C32305C0BC25CE53898
:10556400C394364002800122788E798C7B06E7F65C
:105574001819DBFAA63818A639AA39AB38AE02AF27
:1055840003EEC4035407FEEFC403FF54F84EFEEFCA
:105594005407FF78037989C3E79AFC09E79BFD095F
:1055A40050066304FF6305FFC3EC9EED9F5074D85F
:1055B400E6789679947C06E7F61819DCFAA60318BF
:1055C400A6027991AE02AF03EEC423541FFEEFC4CA
:1055D40023FF54E04EFEEF541FFF7803C3E79AFC09
:1055E40009E79BFD0950066304FF6305FFC3EC9EB6
:1055F400ED9F502FD8E6788F7A007B007C007904E9
:10560400EA26FA08EB36FB08EC3400FCD9F2EC137A
:0D561400FCEB13FBEA13FAEC13EB13F53774
:10562100EA13F536D23A22303A31C23A12565D5077
:105631002A853D3E853C3D853B3C853A3B85073A85
:10564100303913E5406F600EE507B53B0EB53C0BF5
:10565100B53D08B53E0585073FD23B22905778E519
:105661003793FF9056A423232582F582E5833400E6
:10567100F583125683400A0F12568340040F1256C7
:105681008322E493F9A3E493FAA3E493FBA3E493C1
:10569100FCA3C3E5369AE537995007C3EC9536EB81
:1056A100953722EA25DD89DD89D324D324CBD2CBDA
:1056B100D2C4DBC4DBBE39BE39B7CAB7CAB18EB1F9
:1056C1008EAB87AB87A59CA59CA000A0009A969A5B
:1056D1009695D895D891E591E58D858D8588AF888A
:1056E100AF840C840C7F9A7F9A7B497B49771B7727
:1056F1001B730F730F6F276F276B576B5767AB6761
:10570100AB642C642C60C660C65D795D795AFE5A23
:10571100FE5970597057E257E25661566154E75489
:10572100E7537453745207520750A050A04F404F93
:10573100404DE64DE64C934C934B414B4149F54965
:10574100F548B548B547764776463E463E45084555
:1057510008432A432A40E440E43F533F533E3E3E40
:105761003E3C943C943A863A8639183918380500FB
:105771000000000000000032323232323232323266
:1057810032323232323232323232323232323232F8
:1057910032323232323232323232323232323232E8
:1057A10032323232323232323232323232323232D8
:1057B100313130302F2E2D2D2D2C2C2B2A2929281B
:1057C10027262525242323222120201F1E1E1D1CC0
:1057D1001C1B1A1A1A1A191919181818171717173A
:1057E1001616161615151515141414141313131370
:1057F100121212121111111110101010100F0F0F9F
:105801000F0F0E0E0E0E0D0D0D0D0C0C0C0C0B0BC7
:105811000B0B0B0B0A0A0A0A0A09090909090908EB
:105821000808080808070707070707060606060607
:10583100060605050505050504040404040404031E
:105841000303030303030202020202020201010134
:10585100010101010101010101010100000000003C
:105861000000000000000000000000000000000037
:075871000000000000000030
:106E9400C007C0007F01127B8A7F4C127B5B7F544A
:106EA400127B5B7F52127B5B7F20127B5B20490449
:106EB4007F3080027F31127B5B7F20127B5B9001ED
:106EC400E8E0784C127994784C8607430730127BBB
:106ED4005B088607430730127B5B750720127B5BD8
:106EE4009001E9E0784C12798C784C86074307309E
:106EF400127B5B088607430730127B5B08860743D7
:106F04000730127B5B750720127B5B9001EAE07807
:106F14004C127994784C8607430730127B5B0886C1
:106F240007430730127B5B750720127B5BD000D0D0
:106F34000722C007C0007F11127B8A7F4C127B5B43
:106F4400750720127B5B204E047F3080027F311254
:106F54007B5B7F20127B5B9001B2E0784C127994CA
:106F6400784C8607430730127B5B0886074307305B
:106F7400127B5B750720127B5B9001B3E0784C12A7
:106F8400798C784C8607430730127B5B088607436D
:106F94000730127B5B088607430730127B5B75075B
:106FA40020127B5B9001B4E0784C127994784C8683
:106FB40007430730127B5B088607430730127B5B6D
:106FC400750720127B5B9001B5E0784C12799478B8
:106FD4004C8607430730127B5B0886074307301251
:076FE4007B5BD000D0072207
:106BD900003800512372461765340E5F2D7C481921
:106BE9006B3A1C4D3F6E5A0B79281243316054059C
:106BF9007726001F3D227A654758756A48570F1056
:106C0900322D6877554A120D2F301D02203F6778C3
:106C19005A45006245270B694E2C157750321E7C68
:106C29005B39294B6C0E224067053C5E791B375551
:106C3900721052301775593B1C7E472502604C2E45
:106C4900096B7B193E5C701235576E0C2B49650731
:106C59002042264463012D4F680A33517614385A6D
:106C69007D1F0F6D4A28046641231A785F3D117311
:106C79005436741631537F1D3A58610324466A0805
:106C89002F4D5D3F187A56341371482A0D6F4321F1
:106C990006644F2D0A68442601635A381F7D513313
:106CA9001476660423416D0F284A73113654781AF5
:106CB9003D5F1D7F583A16745331086A4D2F0361A1
:106CC9004624345671133F5D7A18214364062A48D5
:106CD9006F0D690B2C4E620027457C1E395B7715B9
:106CE9003250402205674B290E6C553710725E3CB5
:106CF9001B793B597E1C305275172E4C6B09254761
:106D0900600212705735197B5C3E076542200C6E94
:106D1900492B004307440D4E0A49195A1E5D145761
:106D29001350317236753C7F3B78286B2F6C256682
:026D39002261D5
:10823200788276ACA24EE433FFC4333354C0FE904E
:1082420001B4E0FD541F25E04EFE9001B2E0FC5463
:1082520010C4540F4E7881F6EC540FC454F0FE90C3
:1082620001B3E0FC54F0C4540F4E7880F6EC540F86
:10827200C454F0FE9001B5E0FC541EC3134E787F47
:10828200F6EF3395E0FE74D92FF582746B3EF583D9
:10829200E493FFED906BDB93FEEF6EFF9001B2E093
:1082A200906BFB936FFF9001B3E0906C1B936FFF99
:1082B200EC906D1B936F787EF69001B5E030E00490
:0B82C200E64480F6D258787D76282232
:10926A004D756C7469706C65204D617374657273A9
:10927A0000204E6F20427573204D61737465722011
:10928A0020002020202020202020202020202020F4
:03929A0020200091
:108BF90075840130990EC299205109D251D29C78BD
:108C090097760422309845209A0CE5997008C29805
:108C190090023E04F0229001B1E06401702CE54A13
:108C290075F005842056102447F582E43401F58354
:108C3900E599F0D2568010245CF582E43401F5837D
:0D8C4900E599F0C256D257C29822C2982277
:107DBB00758401209803027E9B205319209A13E5AA
:107DCB0099700FD253D254754B0AF54A90023D74F9
:107DDB000FF0C29822209A11E599700D90023D7414
:107DEB000FF090023E740180739001B1E0FF6401CB
:107DFB00702CE54A75F005842056102447F582E473
:107E0B003401F583E599F0D2568010245CF582E4B9
:107E1B003401F583E599F0C256D257C29822EFB4DC
:107E2B00021AAB540556E556AA557002055514F9BE
:107E3B00E5991281D29001B1740380209001B1E0D9
:107E4B00FFB4031CAB540556E556AA5570020555F5
:107E5B0014F9E5991281D29001B17404F0C2982201
:107E6B00EFB404299001E3E0FF04F074BA2FF5821C
:107E7B00E43401F583E599F0C2989001E3E0B4286E
:107E8B00149001E57401F0E49001B1F022C2982244
:067E9B00309902C2992299
:1094540020521E1278C143E740754B0AE4F54A9046
:1094640001B1F0C251D252758401759890C29CF535
:0294740099223B
:108B34009001E4E0705C900206E0FF7025D39001A0
:108B4400B7E094869001B6E094674008E4F0A3741B
:108B540002F0800E9001B7E02428F09001B6E034D2
:108B640000F09001B7E02FFF9001B6E03400FE1250
:108B740072BD900206E024BAF582E43401F583EF75
:108B8400F0900206E004F0E0B42807E4F09001E479
:038B940004F022C8
:10861D009001E5E0607A9001B8E0FEA3E0FFC3941D
:10862D0002EE94005006E49001E5F022900206E07F
:10863D007C002FFFEC3EFE1272BD900206E024BAC4
:10864D00F582E43401F583E0FD6F6017900206E0DA
:10865D00FF9001B9E02FFF9001B8E03400FE1272D7
:10866D007CD255900206E004F0E0B42823E490019A
:10867D00E5F0900206F09001B8E07004A3E064020A
:10868D00700E30550BC255128363128C56128CB27C
:01869D0022BA
:1089FF003051647584019001F9E0B40D0050559029
:108A0F008A15F8282873028A3C028A3F028A42029A
:108A1F008A45028A48028A4B028A4E028A51028A8A
:108A2F0054028A57028A5A028A5D028A600293DBD5
:108A3F000295FC0290AC0291200294D602005E02D5
:108A4F00929D029328029158028FF4029547029447
:088A5F000502955E1295A022AC
:1093DB007897E67024759898754B0AF54A90006358
:1093EB00E0B401079001F97404F022E49001B1F0AC
:0A93FB009001F9E004F01278BB22A3
:0F95FC009001B17401F0C2569001F9E004F02221
:1090AC00900063E01475F005A4B54A15E4B5F01111
:1090BC007598981278C1E49001B1F09001F974049C
:1090CC00F0E54A75F00584AFF0BF010EC257900170
:0B90DC00B17401F09001F9E004F022F3
:10912000E54A75F00584AFF0BF042C20571EE54AD0
:1091300075F00584FF2447F582E43401F583E4F0FB
:10914000745C2FF582E43401F583E4F0E49001B11E
:08915000F09001F9E014F02297
:1094D600900063E075F005A424FDB54A1190005A8A
:0F94E600E0F599E49001B1F09001F9E004F02273
:0D005E0090005BE0F5999001F9E004F022BC
:10929D00900063E0FD75F005A4FFE54AB5071FE4F6
:1092AD00B5F01BEDB414079001F97409F022127892
:0F92BD00BBC256E49001B1F09001F9E004F02239
:10932800E54AB4640E1278C1E49001B1F09001F9F5
:109338007409F0E54A75F00584AFF0BF010EC25715
:0D9348009001B17401F09001F9E004F022F1
:10915800E54A75F00584AFF0BF042C20571EE54A98
:1091680075F00584FF2447F582E43401F583E4F0C3
:10917800745C2FF582E43401F583E4F0E49001B1E6
:08918800F09001F9E014F0225F
:108FF400E54AB465389001E4E0B4012B7554017579
:1090040055017556B6E49001B1F0758401AB540571
:1090140056E556AA557002055514F912818CF59936
:0E9024009001F9E004F0229001F9740CF022A2
:10954700AB54AA55A95612818CF599E49001E2F023
:079557009001F9E004F0228D
:109405009001E2E0FF04F074BA2FF582E43401F52F
:1094150083E0F5999001E2E0D39428400BE49001B4
:09942500E4F09001F9E004F022EA
:10955E00E54AB46911C251C252E4900145F090013E
:07956E00B1F09001F9F022B9
:1095A000C251C252E4F54A900145F09001B1F090E9
:0495B00001F9F022AB
:108D67003053527584019001FAE0B40A00504390E1
:108D77008D7DF8282873028D9B028D9E028DA1029E
:108D87008DA4028DA7028DAA028DAD028DB0028D32
:108D9700B3028DB60292CC0290E70291900295132E
:108DA7000200760293AF028FB30291C80294760253
:068DB70095EB120096226C
:1092CC00E54A7029759898900063E0B4010F127804
:1092DC00C1E49001B1F09001FA7403F0221278BB52
:0E92EC00C256E49001B1F09001FAE004F022C5
:1090E700900063E01475F005A4B54A11E4B5F00DDE
:1090F7007598981278C19001FA7403F022E54A75C1
:10910700F00584AFF0BF0110C257C2569001B17489
:0991170001F09001FAE004F022DD
:10919000E54A75F00584AFF0BF042C20571EE54A60
:1091A00075F00584FF2447F582E43401F583E4F08B
:1091B000745C2FF582E43401F583E4F0E49001B1AE
:0891C000F09001FAE014F02226
:10951300900063E075F005A424FDB54A0E90005A4F
:0C952300E0F599C2569001FAE004F02235
:0D00760090005BE0F5999001FAE004F022A3
:1093AF00900063E0FFB414079001FA7406F022EF07
:1093BF0075F005A4B54A14E4B5F0101278BB90010E
:0C93CF00FAE004F0C256E49001B1F02274
:108FB300E54A75F00584AFF0BF0111C257C2569060
:108FC30001B17401F09001FAE004F022E54AB464BF
:108FD3001F1278BB9001E5E0700B9001B1F0900196
:108FE300FA7408F022E49001B1F09001FA7409F0E8
:018FF300225B
:1091C800E54A75F00584AFF0BF042C20571EE54A28
:1091D80075F00584FF2447F582E43401F583E4F053
:1091E800745C2FF582E43401F583E4F0E49001B176
:0891F800F09001FAE014F022EE
:10947600E54AB4651A7554017555017556B8E490F8
:1094860001E3F09001FA7409F09001B17402F02240
:1095EB00E54AB4690BC253E49001B1F09001FAF073
:0195FB00224D
:0C009600C253E49001B1F09001FAF02296
:108B9700900240E0704090023EE0601B7BFF7A92BB
:108BA700796A12923590023F7414F0900240740172
:108BB700F0E490023EF02220591C90023DE070162E
:108BC7007BFF7A92797B12923590023F7414F09072
:108BD70002407401F022900240E0B4011490023F79
:108BE700E0700E7BFF7A92798C129235E490024006
:028BF700F0226A
:107CBF00789AE6600116900000E0600214F09000E0
:107CCF0001E0600214F0900002E0600214F09000F6
:107CDF000CE0600214F090000AE0600214F09000D3
:107CEF000DE0600214F090000BE0600214F09002BF
:107CFF003DE0600214F0789C16E66003027DBA78CE
:107D0F009C760A789BE6600116900004E0600214EE
:107D1F00F0900005E0600214F0900006E06002149D
:107D2F00F0900008E0600214F0900009E060021487
:107D3F00F078A0E6600116900003E0600214F09066
:107D4F000246E0600214F090023FE0600214F07807
:107D5F009D16E67056789D760A90000EE06002142C
:107D6F00F078A2E61846600708E61618700116901C
:107D7F0001FCE0600214F09001FDE0600214F0904D
:107D8F000201E0600214F0900202E0600214F07849
:107D9F009E16E67016789E760A789F16E6700C7817
:0C7DAF009F7606900200E0600214F022B3
:10958B00C2B59000037405F0900003E06004C2B50F
:05959B0080F6D2B522AC
:1065D100535155452020434F53202053454E534599
:1065E100004F4E202020202020202020202020206D
:1065F10020004F464620202020202020202020203F
:106601002020002020205245504541544552203140
:106611002020200020202052455045415445522041
:10662100322020200020202052455045415445521F
:106631002033202020002020205245504541544540
:106641005220342020200020202052455045415422
:106651004552203520202000202020524550454120
:1066610054455220362020200020202052455045FC
:1066710041544552203720202000202020524550EF
:1066810045415445522038202020002020205245E9
:1066910050454154455220392020200020202052CD
:1066A10045504541544552203130202000202020C2
:1066B100524550454154455220313120200020207F
:1066C100205245504541544552203132202000206E
:1066D100202052455045415445522031332020005D
:1066E100202020524550454154455220313420202C
:1066F100002020205245504541544552203135203B
:106701002000202020524550454154455220313629
:10671100202000202020524550454154455220312F
:106721003720200020202052455045415445522019
:1067310031382020002020205245504541544552F7
:106741002031392020002020205245504541544518
:1067510052203230202000204453502042555320F3
:1067610052657365742020002020454570726F6D5D
:096771002077726F6E6721200091
:10002E00750C01E50CC394155018AF0C74702FF5B8
:10003E0082E43401F583E0FFEF60037F0122050CBB
:04004E0080E17F00CE
:01005200228B
:108D0E00205855127F6FEF6401704D9000A2E0FF66
:108D1E00EF24FF924E9001B0E0FF749A2FF582E49B
:108D2E003401F583E0FF9001B2EFF09001B0E0FF67
:108D3E0074852FF582E43401F583E0FF9001B3EFE3
:108D4E00F09001B0E0FF9001B4EFF01285179001A2
:098D5E00B5EFF0128232D23F227F
:107F6F00900140E4F0A3E4F0900143E4F0A3E4F0C7
:107F7F0090013FE4F090013FE0FFEFC39415400301
:107F8F000280139001B0E0FFEFD3941440069001EC
:107F9F00B07401F09001B0E0FF74702FF582E434FB
:107FAF0001F583E0FF900142EFF0900142E0FFEF17
:107FBF00B401159001B0E0FF74702FF582E4340125
:107FCF00F5837402F07F0122900142E0FFEFB402CB
:107FDF0024900140E0FEA3E0FFEF4E7018900140A7
:107FEF00E4F0A37401F09001B0E0FF7E0090014334
:107FFF00EEF0A3EFF09001B0E004F090013FE00449
:10800F00F0027F84900140E0FEA3E0FFEF4E70048A
:10801F007F002222900144E0FF9001B0EFF07F013A
:01802F00222E
:107EA100900140E4F0A3E4F0900143E4F0A3E4F096
:107EB10090013FE4F090013FE0FFEFC394154003D0
:107EC100027F529001B0E0FFEFD39414400690017D
:107ED100B07401F09001B0E0FF74702FF582E434CA
:107EE10001F583E0FF900142EFF0900142E0FFEFE6
:107EF1006050900063E0FF9001B0E0FEEE6F6042E1
:107F0100900142E0FFEFB401159001B0E0FF747001
:107F11002FF582E43401F5837402F07F0122900190
:107F210040E0FEA3E0FFEF4E70189001B0E0FF7E4D
:107F310000900143EEF0A3EFF0900140E4F0A37450
:107F410001F09001B0E004F090013FE004F0027E06
:107F5100B6900140E0FEA3E0FFEF4E70047F0022E7
:0E7F610022900144E0FF9001B0EFF07F01227A
:10851700900063E0FF74462FF582E43401F583E0B1
:10852700FFEFB4FF06900063E0FF22751D00E51D15
:10853700C39414505BAF1DEF25E024F0F582E434BB
:1085470000F583E0FF900063E0FE74C62EF582E439
:108557003400F583E0FEEEC39F4031AF1DEF25E009
:1085670024EFF582E43400F583E0FF74462FF582AB
:10857700E43401F583E0FFEFB4FF11AF1DEF25E011
:1085870024EFF582E43400F583E0FF22051D809E89
:028597007F0063
:0185990022BF
:10869E00757A00E57AC394145074AF7AEF25E0240E
:1086AE00F0F582E43400F583E0FF900063E0FE74A1
:1086BE00C62EF582E43400F583E0FEEEC39F404AF9
:1086CE00AF7AEF25E024EFF582E43400F583E0FF86
:1086DE0074462FF582E43401F583E0FFEFB4FF2AF0
:1086EE00AF7AEF25E024EFF582E43400F583E0FF66
:1086FE00900063E0FEEF6E6011AF7AEF25E024EF9D
:10870E00F582E43400F583E0FF22057A80857F0050
:01871E002238
:10871F00757B00E57BC394145074AF7BEF25E02489
:10872F0018F582E43401F583E0FF900063E0FE74F6
:10873F00C62EF582E43400F583E0FEEEC39F404A77
:10874F00AF7BEF25E02417F582E43401F583E0FFDA
:10875F0074462FF582E43401F583E0FFEFB4FF2A6E
:10876F00AF7BEF25E02417F582E43401F583E0FFBA
:10877F00900063E0FEEF6E6011AF7BEF25E02417F2
:10878F00F582E43401F583E0FF22057B80857F00CD
:01879F0022B7
:06962E00900063E0FF2242
:10775D009001AFE0FFEFD3941440069001AF740198
:10776D00F090013FE4F09001AFE0FF74852FF582BA
:10777D00E43401F583E0FF9001AFE0FE745B2EF57C
:10778D0082E43401F583E0FEEEB507269001AFE00B
:10779D00FF749A2FF582E43401F583E0FF9001AF79
:1077AD00E0FE74462EF582E43401F583E0FEEE6FC3
:1077BD00600690013F7401F09001AFE0FF74462F19
:1077CD00F582E43401F583E0FF900063E0FEEF6E97
:1077DD00600E900063E0FF9001AFE0FEEE6F703A37
:1077ED0090013FE0FFEF60439001AFE0FFEFD394D6
:1077FD001550149001AFE0FF74702FF582E4340141
:10780D00F5837401F080249001AFE0FF74702FF5C3
:10781D0082E43401F583E4F080119001AFE0FF7450
:10782D00702FF582E43401F583E4F090013FE0FF21
:10783D00EF60449001AFE0FF745B2FF582E43401FB
:10784D00F583E0FF9001AFE0FE74852EF582E43400
:10785D0001F583EFF09001AFE0FF74462FF582E460
:10786D003401F583E0FF9001AFE0FE749A2EF582AE
:0E787D00E43401F583EFF09001AFE004F02257
:106D3B009001EFE0FFEF6003026DED900006E0FFC6
:106D4B00EF70037F0122305D0512789D800312786E
:106D5B00A3204A037F0022128F71EF6401600302AC
:106D6B006DEA304A77C24A126E94900050E0FF9061
:106D7B0001EBEFF0900051E0FF9001ECEFF0900091
:106D8B004FE0FF9001EDEFF09001EDE0FFEFB41F4E
:106D9B00199001E9E0FF9001ECE0FEEEB5070B1254
:106DAB0078A3900006E4F07F01229001E8E0FF90C9
:106DBB0001EBE0FEEEB5070E9001E9E0FF9001EC70
:106DCB00E0FEEE6F60099001EF7401F07F002290FE
:106DDB000094E0FF900006EFF07F00227F00227FFF
:106DEB0000229001EFE0FFEF64016003026E8C90D4
:106DFB000006E0FFEF70037F0122305D0512789DE6
:106E0B0080031278A3204A037F0022C24A126E9499
:106E1B00900050E0FF9001EBEFF0900051E0FF90FD
:106E2B0001ECEFF090004FE0FF9001EDEFF09001DF
:106E3B00EDE0FFEFB41F199001E9E0FF9001ECE0EA
:106E4B00FEEEB5070B1278A3900006E4F07F01224B
:106E5B009001E8E0FF9001EBE0FEEEB5072090011A
:106E6B00E9E0FF9001ECE0FEEEB50712900094E034
:106E7B00FF900006EFF09001EFE4F07F00227F001F
:096E8B00229001EFE4F07F0022E7
:108F710090008BE0FFEF600D1278C740047F018005
:108F8100027F00222290008CE0FFEF601390008DA1
:108F9100E0FFE533D39F40047F0122227F0022229C
:108FA10090008DE0FFE533C39F50047F0122227FB3
:028FB10000229C
:1068F8009001F6E0FFEF60030269B8900008E0FF3E
:10690800EF70037F0122205D0B1278A3900008E44A
:10691800F07F0122128F71EFB4010512789D800378
:106928001278A39001F5E0FFEFB40106203B037F46
:1069380000229001F5E0FFEFB402062041037F003A
:1069480022128F71EF640170649001F5E0FFEF642B
:10695800017021303B1EC23BE540653F6009900154
:10696800F67401F07F0022900099E0FF900008EF94
:10697800F07F00229001F5E0FFEF6402702F3041B4
:106988002CC2419001F8E535F09001F8E0FF900144
:10699800F7E0FEEE6F60099001F67401F07F0022C7
:1069A800900099E0FF900008EFF07F00227F00221E
:1069B8009001F6E0FFEF64016003026A749000083A
:1069C800E0FFEF70037F0122205D101278A3900191
:1069D800F6E4F0900008E4F07F0122128F71EFB422
:1069E800010512789D80031278A39001F5E0FFEF6E
:1069F800B40106203B037F00229001F5E0FFEFB4CD
:106A080002062041037F0022128F71EF6401705A41
:106A18009001F5E0FFEFB4011C303B19C23BE540A3
:106A2800B53F129001F6E4F0900099E0FF9000085D
:106A3800EFF07F00229001F5E0FFEF6402702B3049
:106A48004128C2419001F8E535F09001F8E0FF9047
:106A580001F7E0FEEEB507129001F6E4F090009918
:0D6A6800E0FF900008EFF07F00227F002289
:108A67007BFF7A6579D11292001278C7400B7BFFA2
:108A77007A6579E212923580097BFF7A6579F3127C
:108A870092357F17127B8AAF3312795E90005CE0D4
:108A9700FF127B5B90005DE0FF127B5B90005EE066
:108AA700FF127B5B7F1C127B8AAF3212795E9000CC
:108AB7005CE0FF127B5B90005DE0FF127B5B900048
:078AC7005EE0FF127B5B2261
:10935500900090E0FFEF6013900091E0FFE532D3BD
:109365009F40047F0122227F002222900091E0FF8E
:0D937500E532C39F50047F0122227F0022B9
:1095750090008BE0FFEF60071287A012891C221272
:069585006A75126FEB2273
:1087A0009001FEE0FFEF70161278C7407290008EC5
:1087B000E0FF90000AEFF09001FEE004F02290014B
:1087C000FEE0FFEF640170281278C7401C90000A99
:1087D000E0FFEF704AD25D900098E0FF90000CEF50
:1087E000F09001FEE004F022229001FEE4F022224B
:1087F0009001FEE0FFEFB402211278C7400B900019
:1088000098E0FF90000CEFF02290000CE0FFEF707A
:108810000EC25D9001FEE4F022229001FEE4F022FF
:106A75009001FEE0FFEF704C90008CE0FFEF60238B
:106A850090008DE0FFE533D39F401390008EE0FF2B
:106A950090000AEFF09001FEE004F0228026C25D2E
:106AA50022802190008DE0FFE533C39F50139000B5
:106AB5008EE0FF90000AEFF09001FE7403F0228053
:106AC50003C25D229001FEE0FFEF64017035900086
:106AD5008DE0FFEF24FBFFE533D39F401F90000AB5
:106AE500E0FFEF6003026BD8D25D90008FE0FF906E
:106AF500000CEFF09001FEE004F022229001FEE48C
:106B0500F022229001FEE0FFEF6402702E90008DCE
:106B1500E0FFEF24FBFFE533D39F400B90008FE0B0
:106B2500FF90000CEFF02290000CE0FFEF600302F5
:106B35006BD8C25D9001FEE4F022229001FEE0FFD9
:106B4500EF6403704390008DE0FF7E00EF2405FFA6
:106B5500EE3400FEAD337C00C3ED9FEE6480F8ECAF
:106B6500648098501C90000AE0FFEF7066D25D903B
:106B7500008FE0FF90000CEFF09001FEE004F022A2
:106B8500229001FEE4F022229001FEE0FFEF640472
:106B9500703C90008DE0FF7E00EF2405FFEE340091
:106BA500FEAD337C00C3ED9FEE6480F8EC64809805
:106BB500500B90008FE0FF90000CEFF02290000C3E
:106BC500E0FFEF700EC25D9001FEE4F0222290011D
:046BD500FEE4F022C8
:106FEB009001FFE0FFEF704C90008CE0FFEF60230F
:106FFB0090008DE0FFE533D39F401390008EE0FFB0
:10700B0090000BEFF09001FFE004F0228026C25EAF
:10701B0022802190008DE0FFE533C39F5013900039
:10702B008EE0FF90000BEFF09001FF7403F02280D5
:10703B0003C25E229001FFE0FFEF6401703190000C
:10704B008DE0FFEF24FBFFE533D39F401B90000B3C
:10705B00E0FFEF600302713DD25E90000D7464F0AF
:10706B009001FFE004F022229001FFE4F022229035
:10707B0001FFE0FFEFB4022A90008DE0FFEF24FB4D
:10708B00FFE533D39F400790000D740AF022900068
:10709B000DE0FFEF600302713DC25E9001FFE4F073
:1070AB0022229001FFE0FFEF6403703F90008DE020
:1070BB00FF7E00EF2405FFEE3400FEAD337C00C3F2
:1070CB00ED9FEE6480F8EC648098501890000BE014
:1070DB00FFEF705ED25E90000D7464F09001FFE0E4
:1070EB0004F022229001FFE4F022229001FFE0FF46
:1070FB00EF6404703890008DE0FF7E00EF2405FFF5
:10710B00EE3400FEAD337C00C3ED9FEE6480F8ECF3
:10711B00648098500790000D7464F02290000DE08D
:10712B00FFEF700EC25E9001FFE4F022229001FF90
:03713B00E4F0225B
:10891C009001FFE0FFEF70161278C7406A90008E4E
:10892C00E0FF90000BEFF09001FFE004F0229001CB
:10893C00FFE0FFEF640170241278C7401890000B21
:10894C00E0FFEF7042D25E90000D7464F09001FF76
:10895C00E004F022229001FFE4F022229001FFE0DB
:10896C00FFEFB4021D1278C7400790000D7464F03D
:10897C002290000DE0FFEF700EC25E9001FFE4F05C
:08898C0022229001FFE4F02219
:10952F0012871F8F7C900245E0FFEF657C600890EB
:07953F000245E57CF0D25F5C
:019546002202
:1079A700900063E0FFEF12820C79F00179FA027A16
:1079B70004037A0E047A18057A22067A2C077A3697
:1079C700087A40097A4A0A7A540B7A5E0C7A680D6B
:1079D7007A720E7A7C0F7A86107A90117A9A127AD6
:1079E700A4137AAE1400007AB77BFF7A6679041283
:1079F7009235227BFF7A667915129235227BFF7AC0
:107A0700667926129235227BFF7A6679371292358C
:107A1700227BFF7A667948129235227BFF7A667954
:107A270059129235227BFF7A66796A129235227B48
:107A3700FF7A66797B129235227BFF7A66798C1200
:107A47009235227BFF7A66799D129235227BFF7AE7
:107A57006679AE129235227BFF7A6679BF1292352C
:107A6700227BFF7A6679D0129235227BFF7A66797C
:107A7700E1129235227BFF7A6679F2129235227BE8
:107A8700FF7A677903129235227BFF7A677914129E
:107A97009235227BFF7A677925129235227BFF7A0E
:107AA700677936129235227BFF7A677947129235CA
:017AB70022AC
:10942E00900202E0FFEF701D7BFF7A67795812926F
:10943E0000900003740AF0900003E0FFEF70F875DF
:06944E00840075EF03220B
:10622700757500757409D3E5746480948640677545
:106237007313C3E573648094804057AF73EF33954E
:10624700E0FE74C72FF58274003EF583E0FFEF652B
:1062570074703BE57304FFAE75EE25E024EFF5821D
:10626700E43400F583EFF0AF75EF25E024F0F58215
:10627700E43400F583E574F00575E575D3941440AF
:106287000D7BFF7A677969129200D26080041573DB
:1062970080A015748090757406D3E574648094802B
:1062A7004067757300C3E573648094945057AF7368
:1062B700EF3395E0FE74C72FF58274003EF583E057
:1062C700FFEF6574703BE57304FFAE75EE25E024C0
:1062D700EFF582E43400F583EFF0AF75EF25E024A6
:1062E700F0F582E43400F583E574F00575E575D3C0
:1062F7009414400D7BFF7A677969129200D260800F
:1063070004057380A015748090E5756414600B7B99
:10631700FF7A677969129200D26075750075740902
:10632700D3E574648094864067757300C3E573642E
:106337008094945057AF73EF3395E0FE74C72FF5F1
:106347008274003EF583E0FFEF6574703BE57304EC
:10635700FFAE75EE25E02417F582E43401F583EFEF
:10636700F0AF75EF25E02418F582E43401F583E5F5
:1063770074F00575E575D39414400D7BFF7A677942
:1063870069129200D2608004057380A01574809012
:10639700757406D3E574648094804067757313C37E
:1063A700E573648094804057AF73EF3395E0FE74D4
:1063B700C72FF58274003EF583E0FFEF6574703BED
:1063C700E57304FFAE75EE25E02417F582E434018A
:1063D700F583EFF0AF75EF25E02418F582E434017B
:1063E700F583E574F00575E575D39414400D7BFFCF
:1063F7007A677969129200D2608004157380A015BC
:10640700748090E5756414600B7BFF7A6779691275
:046417009200D260BD
:01641B00225E
:104AE3002020464C4558495620303038432020205A
:104AF30000527074724E756D62657257726F6E6795
:104B0300210050726F6772616D6D696E67526573D4
:104B13006574002049502050524F4752414D4D4932
:104B23004E47200043544353532036332E30202026
:104B33002020202043544353532036372E30202047
:104B43002020202043544353532036392E34202031
:104B53002020202043544353532037312E39202023
:104B63002020202043544353532037342E34202015
:104B73002020202043544353532037372E30202006
:104B83002020202043544353532037392E372020ED
:104B93002020202043544353532038322E352020E5
:104BA3002020202043544353532038352E342020D3
:104BB3002020202043544353532038382E352020BF
:104BC3002020202043544353532039312E352020B5
:104BD3002020202043544353532039342E3820209F
:104BE3002020202043544353532039372E34202090
:104BF300202020204354435353203130302E302083
:104C0300202020204354435353203130332E35206A
:104C1300202020204354435353203130372E322059
:104C2300202020204354435353203131302E392048
:104C3300202020204354435353203131342E382035
:104C4300202020204354435353203131382E382021
:104C5300202020204354435353203132332E30201D
:104C6300202020204354435353203132372E332006
:104C7300202020204354435353203133312E3820F6
:104C8300202020204354435353203133362E3520E4
:104C9300202020204354435353203134312E3320DA
:104CA300202020204354435353203134362E3220C6
:104CB300202020204354435353203135312E3420B8
:104CC300202020204354435353203135362E3720A0
:104CD300202020204354435353203135392E38208C
:104CE300202020204354435353203136322E322088
:104CF300202020204354435353203136352E352072
:104D0300202020204354435353203136372E39205B
:104D1300202020204354435353203137312E332056
:104D2300202020204354435353203137332E38203F
:104D3300202020204354435353203137372E332030
:104D4300202020204354435353203137392E392018
:104D5300202020204354435353203138332E352011
:104D6300202020204354435353203138362E322001
:104D7300202020204354435353203138392E3920E7
:104D8300202020204354435353203139322E3820DE
:104D9300202020204354435353203139362E3620CC
:104DA300202020204354435353203139392E3520BA
:104DB300202020204354435353203230332E3520B8
:104DC300202020204354435353203230362E3520A5
:104DD300202020204354435353203231302E372098
:104DE300202020204354435353203231382E312086
:104DF300202020204354435353203232352E372072
:104E0300202020204354435353203232392E312063
:104E1300202020204354435353203233332E362053
:104E2300202020204354435353203234312E382042
:104E3300202020204354435353203235302E332037
:104E4300202020204354435353203235342E312025
:104E5300202020202020202020202020202020204F
:044E630020202020CB
:10602A0075840F12641C12960B7BFF7A4A79E3126D
:10603A00920012789D20A10875840F43E8C080065B
:10604A0075840F53E83F12958B9000037401F0900A
:10605A000003E070FA9002477401F090024874035A
:10606A00F07D007CFC7F1012906FE4900247F09064
:10607A000248F0C2601295D9900063E0FF6005D330
:10608A00941440119000637401F07BFF7A4A79F40A
:10609A00129200D2602060121279A7128363128CC6
:1060AA0056128CB21292FA126227900202740FF000
:1060BA001278911278B59000A1E0FF78A1760008D5
:1060CA00A6079000ACE0900200F0E4900145F09041
:1060DA0001E7F09001E6F09001EFF09001F9F090FD
:1060EA00005A74FFF090005BF0E4900245F09002D1
:1060FA0044F0F559C265C262C2631278A390023DA8
:10610A00740FF030431312431F1295D9128363128E
:10611A008C56128CB2C24380EA20A60E128A67E419
:10612A009001E7F09001E6F080EF30461DC246127A
:10613A00431F1295D9128363128C56128CB212968F
:10614A000BE49001E6F09001E7F043E7403059068E
:10615A00128B3412945430A704C2A78002D2A71219
:10616A003EAB122FF312713EE55CB4551DE55DB4EA
:10617A00AA189002467414F0900246E070FA7BFF67
:10618A007A4B79051292001278971278A9503E122A
:10619A00942E1274F512775D125628129575128B89
:1061AA009712952F305F1E20621BC25F900245E056
:1061BA002400FEE4341790021DF0A3CEF0900219D9
:1061CA007401F0D262E490024BF0026123127891DA
:1061DA009000BCE060031278B59000A1E0FF78A1BE
:1061EA00760008A6079000ACE0900200F0E4900167
:1061FA00E7F09001E6F09001EFF0900063E0900084
:10620A005AF090005B74FCF01278A3900202741E9C
:0D621A00F07BFF7A4B791612677A02612340
:108ACE0001AE01C901DA01EB01FC020E02200233F4
:108ADE000247025C02710287029902AB02C302DCFA
:108AEE0002F50310032B03480365038403A403C597
:108AFE0003E6040A042E04430453046A047A049120
:108B0E0004A204BA04CC04E504F705100524053EBE
:108B1E000552056D0582059E05D10605061C063B10
:068B2E00067306AD06C748
:1094F500C23DC23FEF25E024CEF582E4348AF583F0
:0E950500E493F51A740193F51BD23ED238227E
:09962500C23DC23FC23EC2382220
:0300A300028F2E9B
:108F2E00C0E0C0F0C083C082C0D075D000C000C009
:108F3E0001C002C003C004C005C006C00720590509
:108F4E00127DBB8003128BF9D007D006D005D0045A
:108F5E00D003D002D001D000D0D0D082D083D0F0B8
:038F6E00D0E0321E
:030093000289944B
:0B899400C0E0C0D075D000C006C007D6
:10899F00AE84758402E5347007AFBE75BB07802FB8
:1089AF00E534B40107AFBE75BB048023E534B402D0
:1089BF0007AFBE75BB068017E534B4030885BE321A
:1089CF0075BB04800AE534B40409AFBE75BB050559
:1089DF00348010E534B4050885BE3375BB048000C0
:0789EF00753400C2ED8E8417
:0989F600D007D006D0D0D0E03249
:03008300029032B6
:10903200C0E0C0F0C083C082C0D075D000C000C004
:1090420001C002C003C004C005C006C007C2CF12DF
:109052001F95D007D006D005D004D003D002D0018E
:0D906200D000D0D0D082D083D0F0D0E0324A
:030073000284877D
:10848700C0E0C0F0C083C082C0D075D000C000C0BB
:1084970001C002C003C004C005C006C007C2CF3078
:1084A70059051289FF8003128D677897E6600116D8
:1084B700304027C240D54B05754B0A054A1273B9A0
:1084C700D51C09751C0A758401438820D5311B7595
:1084D70031607584024388208010D2401276D378A9
:1084E7009816E670057604121BC37584014388103D
:1084F700758402D2ECD007D006D005D004D003D0C3
:1085070002D001D000D0D0D082D083D0F0D0E032DA
:03006B00028E5DA5
:108E5D00C0E0C0F0C083C082C0D075D000C000C0DB
:0D8E6D0001C002C003C004C005C006C0075C
:0E8E7A0085846F127CBF758402C28D856F8463
:108E8800D007D006D005D004D003D002D001D0003E
:0B8E9800D0D0D082D083D0F0D0E032E8
:03005B00028E0F03
:108E0F00C0E0C0F0C083C082C0D075D000C000C029
:108E1F0001C002C003C004C005C006C00712555DE3
:108E2F007899E6600116900007E0600214F07584EF
:108E3F0001C28DD007D006D005D004D003D002D008
:0E8E4F0001D000D0D0D082D083D0F0D0E0325D
:03005300028EA377
:108EA300C0E0C0F0C083C082C0D075D000C000C095
:108EB30001C002C003C004C005C006C007C28C3095
:108EC3005B04C25B8005D25B1273DBD007D006D094
:108ED30005D004D003D002D001D000D0D0D082D0AE
:068EE30083D0F0D0E03264
:03002B00020016BA
:03001600C2CF3224
:030023000295C77C
:1095C700309904C299C267309807859957C298D2D3
:0295D7006632FA
:03001B00020019C7
:0100190032B4
:108EE900A984A2AF9268AEB1C2AF75840F53A1FE37
:108EF9008FB1E4F584900247E042B7900248E0421E
:108F09008F8C088D098D828C83EBF0E4F5849002B7
:108F190048E0F4528F900247E0F452B78EB1898449
:048F2900A26892AFF9
:018F2D002221
:10906F00A984A2AF9268AEB1C2AF8C088D098FB13F
:10907F00E4F584900247E0FF42B7E4F5849002489C
:10908F00E0FD428F850982850883E4F0EDF4528F6D
:0C909F00EFF452B78EB18984A26892AF42
:0190AB0022A2
:10949600AE84A2AF9268ABB1C2AF8FB18C0A8D0B0E
:0F94A6008D828C83E493FF8BB18E84A26892AF8A
:0194B5002294
:100EC800202020464C45582049562020202020200C
:100ED8000020202020202020202020202049444CB1
:100EE80045002054657374696E67204D6F646520F2
:100EF80020200043726F7373204275737920434F2B
:100F08005320200043726F73732042757379205306
:100F1800454E53450053656E642049646C654D65C4
:100F28007373616765002020474F544F204D455328
:100F380053414745202000202053656E64696E6741
:100F48002043574944202000204357494420554412
:100F5800544420464C414720004453502046494EB3
:100F68004953485320435749440031335741495462
:100F7800205544544420464C41470032315741499A
:100F880054205544544420464C414700333357417C
:100F98004954205544544420464C41470033375760
:100FA800414954205544544420464C4147004C5430
:100FB80052564F4950204F5554474F494E470034D9
:100FC8003457414954205544544420464C41470025
:100FD800343857414954205544544420464C4147DD
:100FE80000353057414954205544544420464C411B
:100FF8004700204C6F63616C2048616E672054691C
:101008006D650035335741495420554454442046B2
:101018004C41470057616974204361727269657277
:1010280044726F7000353757414954205544544431
:1010380020464C41470020564F4950204F555447B1
:101048004F494E4720200020564F49502048616E96
:10105800672054696D65200020576169744E657476
:10106800776F726B48616E67003633574149542079
:101078005544544420464C4147003637574149545B
:10108800205544544420464C414700373057414985
:1010980054205544544420464C4147002020494E92
:1010A800434F4D494E47204C545220200037335768
:1010B800414954205544544420464C414700373850
:1010C80057414954205544544420464C4147003820
:1010D8003057414954205544544420464C41470018
:1010E8002020494E434F4D494E47204354435353C4
:1010F8002020002020494E434F4D494E472044436D
:101108005320200038345741495420554454442032
:10111800464C4147003838574149542055445444B7
:1011280020464C41470043726F73732042757379B0
:10113800204D6F6465310043726F7373204275737D
:1011480079204D6F6465320043726F737320427566
:101158007379204D6F6465330043726F7373204257
:10116800757379204D6F646534003933574149549C
:10117800205544544420464C41470043544353535C
:101188002036332E30202020202020435443535330
:101198002036372E3020202020202043544353531C
:1011A8002036392E34202020202020435443535306
:1011B8002037312E392020202020204354435353F8
:1011C8002037342E342020202020204354435353EA
:1011D8002037372E302020202020204354435353DB
:1011E8002037392E372020202020204354435353C2
:1011F8002038322E352020202020204354435353BA
:101208002038352E342020202020204354435353A7
:101218002038382E35202020202020435443535393
:101228002039312E35202020202020435443535389
:101238002039342E38202020202020435443535373
:101248002039372E34202020202020435443535364
:10125800203130302E302020202020435443535357
:10126800203130332E35202020202043544353533F
:10127800203130372E32202020202043544353532E
:10128800203131302E39202020202043544353531D
:10129800203131342E38202020202043544353530A
:1012A800203131382E3820202020204354435353F6
:1012B800203132332E3020202020204354435353F2
:1012C800203132372E3320202020204354435353DB
:1012D800203133312E3820202020204354435353CB
:1012E800203133362E3520202020204354435353B9
:1012F800203134312E3320202020204354435353AF
:10130800203134362E32202020202043544353539A
:10131800203135312E34202020202043544353538C
:10132800203135362E372020202020435443535374
:10133800203135392E382020202020435443535360
:10134800203136322E32202020202043544353535C
:10135800203136352E352020202020435443535346
:10136800203136372E392020202020435443535330
:10137800203137312E33202020202043544353532B
:10138800203137332E382020202020435443535314
:10139800203137372E332020202020435443535305
:1013A800203137392E3920202020204354435353ED
:1013B800203138332E3520202020204354435353E6
:1013C800203138362E3220202020204354435353D6
:1013D800203138392E3920202020204354435353BC
:1013E800203139322E3820202020204354435353B3
:1013F800203139362E3620202020204354435353A1
:10140800203139392E35202020202043544353538E
:10141800203230332E35202020202043544353538C
:10142800203230362E352020202020435443535379
:10143800203231302E37202020202043544353536C
:10144800203231382E31202020202043544353535A
:10145800203232352E372020202020435443535346
:10146800203232392E312020202020435443535338
:10147800203233332E362020202020435443535328
:10148800203234312E382020202020435443535317
:10149800203235302E33202020202043544353530C
:1014A800203235342E3120202020202020202020DA
:1014B800202020202020202020202044435320309A
:1014C800303620494E5620303231204443532030A4
:1014D800303720494E56203231342044435320308F
:1014E800313520494E562031343120444353203081
:1014F800313720494E562030353020444353203070
:10150800323120494E562030303620444353203063
:10151800323320494E56203034372044435320304C
:10152800323520494E56203234342044435320303B
:10153800323620494E562034363420444353203026
:10154800333120494E562036323720444353203019
:10155800333220494E562030353120444353203011
:10156800333620494E5620313732204443532030F9
:10157800343320494E5620343435204443532030E8
:10158800343720494E5620303233204443532030DC
:10159800353020494E5620303137204443532030CF
:1015A800353120494E5620303332204443532030C1
:1015B800353320494E5620343532204443532030A9
:1015C800353420494E56203431332044435320309B
:1015D800363520494E562032373120444353203087
:1015E800373120494E56203330362044435320307B
:1015F800373220494E562032343520444353203068
:10160800373320494E562035303620444353203056
:10161800373420494E562031373420444353203143
:10162800313420494E56203731322044435320313B
:10163800313520494E56203135322044435320312C
:10164800313620494E562037353420444353203113
:10165800323220494E56203232352044435320310D
:10166800323520494E5620333635204443532031F5
:10167800333120494E5620333634204443532031E9
:10168800333220494E5620353436204443532031D6
:10169800333420494E5620323233204443532031CC
:1016A800343120494E5620303135204443532031BF
:1016B800343320494E5620343132204443532031AC
:1016C800343520494E562032373420444353203194
:1016D800353220494E56203131352044435320318C
:1016E800353520494E562037333120444353203175
:1016F800353620494E562032363520444353203162
:10170800363220494E562035303320444353203159
:10171800363520494E562032353120444353203146
:10172800373220494E562030333620444353203137
:10173800373420494E562030373420444353203222
:10174800303520494E562032363320444353203218
:10175800313220494E562033353620444353203207
:10176800313420494E5620303037204443532032FC
:10177800323320494E5620313334204443532032EB
:10178800323520494E5620313232204443532032DC
:10179800323620494E5620343131204443532032CA
:1017A800343320494E5620333531204443532032B8
:1017B800343420494E5620303235204443532032A9
:1017C800343520494E562030373220444353203296
:1017D800343620494E562035323320444353203284
:1017E800353120494E562031363520444353203276
:1017F800353220494E562034363220444353203265
:10180800353520494E56203434362044435320324F
:10181800363120494E562037333220444353203244
:10182800363320494E562032303520444353203237
:10183800363520494E562031353620444353203220
:10184800363620494E56203435342044435320320E
:10185800373120494E562030363520444353203204
:10186800373420494E5620313435204443532033F1
:10187800303620494E5620303731204443532033E8
:10188800313120494E5620363634204443532033D4
:10189800313520494E5620343233204443532033C7
:1018A800323520494E5620353236204443532033B2
:1018B800333120494E5620343635204443532033A3
:1018C800333220494E562034353520444353203393
:1018D800343320494E562035333220444353203385
:1018E800343620494E562036313220444353203373
:1018F800353120494E562032343320444353203367
:10190800353620494E562032313220444353203355
:10191800363420494E562031333120444353203346
:10192800363520494E562031323520444353203332
:10193800373120494E56203733342044435320341E
:10194800313120494E562032323620444353203418
:10195800313220494E562031343320444353203409
:10196800313320494E5620303534204443532034F7
:10197800323320494E5620333135204443532034E6
:10198800333120494E5620373233204443532034D4
:10199800333220494E5620353136204443532034C3
:1019A800343520494E5620303433204443532034B4
:1019B800343620494E56203235352044435320349E
:1019C800353220494E562030353320444353203495
:1019D800353420494E56203236362044435320347D
:1019E800353520494E562033333220444353203472
:1019F800363220494E562032353220444353203463
:101A0800363420494E562030323620444353203451
:101A1800363520494E562033333120444353203441
:101A2800363620494E562036363220444353203528
:101A3800303320494E562031363220444353203526
:101A4800303620494E562030373320444353203512
:101A5800313620494E562034333220444353203502
:101A6800323320494E5620323436204443532035F1
:101A7800323620494E5620333235204443532035E0
:101A8800333220494E5620333433204443532035D3
:101A9800343620494E5620313332204443532035C2
:101AA800363520494E5620373033204443532036AC
:101AB800303620494E5620363331204443532036A1
:101AC800313220494E562033343620444353203691
:101AD800323420494E562036333220444353203680
:101AE800323720494E562030333120444353203674
:101AF800333120494E562036303620444353203661
:101B0800333220494E56203632342044435320364F
:101B1800353420494E562037343320444353203639
:101B2800363220494E562034363620444353203628
:101B3800363420494E562033313120444353203720
:101B4800303320494E56203536352044435320370C
:101B5800313220494E562031313420444353203706
:101B6800323320494E5620343331204443532037F2
:101B7800333120494E5620313535204443532037E0
:101B8800333220494E5620323631204443532037D1
:101B9800333420494E5620333731204443532037BD
:101BA800343320494E5620363534204443532037A9
:0B1BB800353420494E562031313620D4
:1074F50030600302762B9000BBE0FFB4010A9000D8
:107505005A74FFF0E40275D1EF640260030275D688
:1075150012788B9000BCE060031278AF787DE6604E
:10752500030275C53058030275C59001EEE070324F
:10753500D23F9000A2E024FF924E900063E0FF90BE
:1075450001B2F09000A0E09001B3F09001B4EFF02B
:1075550012869E9001B5EFF01282329001EE740210
:10756500F022127EA1EF64017050D23F9001B2E08B
:1075750024DAF582E43400F583E024FF924E90018D
:10758500B0E0FF249AF582E43401F583E09001B27E
:10759500F074852FF582E43401F583E09001B3F0B2
:1075A5009001B0E09001B4F01285179001B5EFF0AD
:1075B5001282329001EEE014F0229001EEE014F018
:1075C500900063E090005AF09000A0E090005BF01E
:1075D500229001E6E0B40A0050439075E6F82828A9
:1075E5007302760402760702760A02760D02761099
:1075F50002761302761602761902761C02761F02AF
:10760500289A0280E10283F60251DF023582024E9A
:1076150067025878023A18024730025BA9E49001E4
:07762500E6F09001E7F022FE
:10289A009001E7E0B40B004003022F719028ADF8D5
:1028AA002828730228CE02290A022B4C022B8C02FA
:1028BA002BAB022BCD022C98022D22022DB8022D11
:1028CA00D6022EC2E4900244F0900241F0C2397B53
:1028DA00FF7A0E79C81292007BFF7A0E79D912928A
:1028EA003590005A74FFF090005BF01278919000D6
:1028FA00BCE060031278B59001E77401F0022F760C
:10290A0020A55F12788B9000BCE060031278AF902C
:10291A0000B9E0900000F0900063E0FF90005AF0E8
:10292A009000A0E0FE90005BF09001E77405F09043
:10293A0001B2EFF09001B3EEF0900063E09001B4C1
:10294A00F01285179001B5EFF09000A2E024FF92F3
:10295A004E128232D23F7BFF7A0E79EA129200023D
:10296A002F76305D60304A5DC24A900050E0FFC366
:10297A009415505174DA2FF582E43400F583E0FFA0
:10298A00A248E4336F703EA2489249900050E0900A
:10299A0001E8F0900051E09001E9F090004FE090DA
:1029AA0001EAF0126E949001EAE0641F6017900148
:1029BA00E8E0FF9001E9E0FD7C001282CD9001E69B
:1029CA007402022DD2C24A12002EBF011712788B4E
:1029DA009000BCE060031278AF9000B9E09000006C
:1029EA00F0022D9E9000BDE0FF64016004EFB40286
:1029FA000B305D087BFF7A0E79FB80199000BDE0F1
:102A0A00FF64036004EFB4041F129355BF01197BDE
:102A1A00FF7A0F790C12920090009AE078A0F69053
:102A2A0001E77409F0022F76128F71EF6401706565
:102A3A00303B28C23B9001F504F0D239853F40E58E
:102A4A004075F010A42483F9741135F0FA7BFF1253
:102A5A009200AF4012889FC239802A304137C24162
:102A6A009001F7E535F075F010A424C3F974143514
:102A7A00F0FA7BFF1292009001F7E0FF12859A901C
:102A8A0001F57402F09001E7740AF090009AE07878
:102A9A00A0F6022F76C23BC24178A2E61846703FE2
:102AAA009000A1E060397BFF7A0F791D12920090A5
:102ABA0000A1E0FF78A1760008A60790005A74FFEB
:102ACA00F090005BF012788B9000BCE06003127803
:102ADA00AF9000B9E0900000F09001E7022F259036
:102AEA0000ACE0FF7003022F76900200E060030260
:102AFA002F769000AAE0FE60107003022F769001F4
:102B0A00FBE064016003022F76900200EFF0E4908C
:102B1A0001FBF012788B9000BCE060031278AF9052
:102B2A0000B9E0900000F0900063E090005AF09045
:102B3A00005B74FDF0E49001E7F09001E604F00216
:102B4A002F76900000E06003022F76305803022FA0
:102B5A0076900063E0FF9001B2F09001B374FFF049
:102B6A009001B4EFF09001B5F09000A2E024FF923A
:102B7A004E128232D23F126F369001E77403F0028E
:102B8A002F76787DE66003022F76305803022F767F
:102B9A00900095E0900001F09001E77404F0022F94
:102BAA0076900001E06003022F761278919000BCC3
:102BBA00E060031278B5E49001E7F09001FB04F0BD
:102BCA00022F7630A503022F2A900063E090005A64
:102BDA00F09000A0E090005BF0128F71BF01051227
:102BEA00789D80031278A3787DE66003022F763001
:102BFA005803022F769001EEE07037D23F9000A280
:102C0A00E024FF924E900063E0FF9001B2F0900042
:102C1A00A0E09001B3F09001B4EFF012869E90010B
:102C2A00B5EFF01282329001EE7402F0126F3602A2
:102C3A002F76127EA1EF6401704BD23F9001B0E073
:102C4A00FF249AF582E43401F583E09001B2F0742E
:102C5A00852FF582E43401F583E09001B3F0900109
:102C6A00B0E09001B4F01285179001B5EFF0900131
:102C7A00B2E024DAF582E43400F583E024FF924ED0
:102C8A0012823280009001EEE014F0022F7690005A
:102C9A0000E06003022F76305803022F76787DE633
:102CAA006003022F7690005A74FFF090005BF012D6
:102CBA007F6FEF64016003022DA79001B0E0FF244B
:102CCA009AF582E43401F583E09001B2F074852F1D
:102CDA00F582E43401F583E09001B3F09001B0E0AD
:102CEA009001B4F012962E9001B5EFF09001B2E087
:102CFA0024DAF582E43400F583E024FF924E12824E
:102D0A0032D23F7BFF7A0F792E129200126F3690E1
:102D1A0001E77407F0022F76305D63304A62C24AD7
:102D2A00900050E0FFC39415505674DA2FF582E4F0
:102D3A003400F583E0FFA248E4336F7043A248925F
:102D4A0049900050E09001E8F0900051E09001E9CC
:102D5A00F090004FE09001EAF0126E949001EAE0E0
:102D6A00641F601C9001E8E0FF9001E9E0FD7C002F
:102D7A001282CDE49001E7F09001E6022F25C24AC3
:102D8A00787DE66003022F76305803022F76120010
:102D9A002EEF60099001E77406F0022F76900095F5
:102DAA00E0900001F09001E77408F0022F7690009D
:102DBA0001E06003022F761278919000BCE0600374
:102DCA001278B59001FB7401F0022F71305D633007
:102DDA004A60C24A900050E0FFC39415505474DA16
:102DEA002FF582E43400F583E0FFA248E4336F70E4
:102DFA0041A2489249900050E09001E8F0900051B9
:102E0A00E09001E9F090004FE09001EAF0126E9430
:102E1A009001EAE0641F601A9001E8E0FF9001E97E
:102E2A00E0FD7C001282CDE49001E7F09001E60219
:102E3A002F25C24A9000BDE0FF64016004EFB4028E
:102E4A000A205D079001E77401F022EF6403600431
:102E5A00EFB4040C129355EF70069001E704F022C8
:102E6A0078A0E66003022F76900063E090005AF0A3
:102E7A0090005B74FDF09000BDE0FF64016004EF18
:102E8A00B40205305D02801C9000BDE0FF6403605F
:102E9A0008EF64046003022F76129355EF64016011
:102EAA0003022F7690009BE0900005F0E49001E782
:102EBA00F09001E67409F022128F71EF64017060DC
:102ECA00304A5FC24A900050E0FFC39415505374D1
:102EDA00DA2FF582E43400F583E0FFA248E4336F89
:102EEA007040A2489249900050E09001E8F09000AA
:102EFA0051E09001E9F090004FE09001EAF0126E83
:102F0A00949001EAE0641F60199001E8E0FF9001E3
:102F1A00E9E0FD7C001282CD9001E67402F0804C5B
:102F2A008045C24A78A0E67043305D40900066E072
:102F3A007004C239803212788B9000BCE0600312B0
:102F4A0078AF12789D9000B9E0900000F09000638D
:102F5A00E090005AF090005B74FEF0E49001E7F014
:102F6A009001E67405F022E49001E7F0900241E056
:102F7A006403704112788B9000BCE060031278AF52
:102F8A009000B9E0900000F0E4900241F090024213
:102F9A00E0FF90005AF0900243E0FE90005BF09050
:102FAA0001E8EFF09001E9EEF0E49001E7F090011A
:102FBA00E67407F022900241E0602D12788B9000AF
:102FCA00BCE060031278AF9000B9E0900000F09086
:102FDA000063E090005AF090005B74FEF0E4900108
:092FEA00E7F09001E67408F02202
:1080E100128D0E9001E7E0702C20622190021D7428
:1080F10018F0A37402F090021914F0D2629001E713
:10810100F07BFF7A0F793F129200027BB37BFF7AFB
:108111000F795080699001E7E0B40120900244E0BA
:1081210064017066F0900095E0900001F09001E725
:108131007402F07BFF7A0F79610292009001E7E00F
:10814100B40219900001E070411278919000BCE0F6
:1081510060031278B59001E77403F0229001E7E023
:10816100B4031E20621290021D7418F0A3E4F09073
:10817100021904F0D26280097BFF7A0F79720292B0
:0B81810035E49001E6F09001E7F022E9
:1083F6009001E7E0703B900070E0602B12788B9064
:1084060000BCE060031278AF9000B9E0900000F085
:108416009001E8E090005AF09001E9E090005BF0EE
:108426009001E77401F022E49001E7F09001E6F094
:10843600229001E7E06401703E2062329001E8E09C
:10844600FE9001E9E07C002400FFEC3E90021DF066
:10845600A3EFF09002197401F0D262900071E090DF
:1084660001E66004740480027403F0E4800E7BFF6E
:108476007A0F7983029235E49001E6F09001E7F0F5
:0184860022D3
:1051DF009001E7E0704A900000E06003025543A29F
:1051EF0049924E9001E8E09001B2F09001E9E09011
:1051FF0001B3F0900063E09001B4F012869E90012D
:10520F00B5EFF0128232D23F126F369001EE740872
:10521F00F0900094E0900006F09001E77401F02206
:10522F009001E7E06401703E126D3BEF6002805524
:10523F00787DE660030255433058030255437628C4
:10524F00D2589001EEE014F0E0600302554374026F
:10525F00F0900094E0900006F0900096E090000E21
:10526F00F09001E7806C9001E7E064026003025365
:10527F003F126D3BEF6002800C900096E060109043
:10528F00000EE0700A1278A39001E77403F0227801
:10529F007DE660030255433058030255439001EEFB
:1052AF00E07033A249924E9001E8E09001B2F09085
:1052BF0001E9E09001B3F0900063E09001B4F012C7
:1052CF00869E9001B5EFF0128232D23F126F369068
:1052DF0001EE7402F022127EA1EF6401704F900173
:1052EF00B0E0FF249AF582E43401F583E09001B237
:1052FF00F074852FF582E43401F583E09001B3F06B
:10530F009001B0E09001B4F01285179001B5EFF065
:10531F009001B2E024DAF582E43400F583E024FF53
:10532F00924E128232D23F126F360253EF0253EF78
:10533F009001E7E0B4032C20622090021DE4F0A35B
:10534F0074FFF09002197401F0D2621278A3E49006
:10535F0001EFF09001E77404F0227BFF7A0F79944C
:10536F000255299001E7E064047043787DE66003FD
:10537F00025543305803025543A249924E9001E81B
:10538F00E09001B2F09001E9E09001B3F09001B428
:10539F00741FF012962E9001B5EFF0128232900129
:1053AF00EE7403F0126F369001E77405F02290014E
:1053BF00E7E0FF64057030787DE660030255433007
:1053CF0058030255439001EEE0700F900095E09066
:1053DF000001F09001E77406F022787D7628D2580C
:1053EF009001EEE014F022EF640660030254EE30F9
:1053FF005D78304A75C24A900050E0FFC394155053
:10540F006974DA2FF582E43400F583E0FFA248E4F3
:10541F00336F7056A2489249900050E09001E8F027
:10542F00900051E09001E9F090004FE09001EAF018
:10543F00641F60369001E8E0FFC39415502C74DAB6
:10544F002FF582E43400F583E0FFA249E433B5077A
:10545F00199001E8E0FF9001E9E0FD7C001282CD98
:10546F009001E67402F0E402551EC24A787DE670A0
:10547F0055205852127F6FEF6401704A9001B0E0CF
:10548F00FF249AF582E43401F583E09001B2F074C1
:10549F00852FF582E43401F583E09001B3F090019C
:1054AF00B0E09001B4F01285179001B5EFF09001C4
:1054BF00B2E024DAF582E43400F583E024FF924E63
:1054CF00128232126F36900001E07068127891905C
:1054DF0000BCE060031278B59001E77407F02290EA
:1054EF0001E7E06407703620622A90021D7418F0FD
:1054FF00A3E4F090021904F0D2629001FBF0900047
:10550F00A1E0FF78A1760008A607E49001E6F090ED
:10551F0001E7F0227BFF7A0F79A50292359001E720
:10552F00E0D39407400EE49001E6F09001E7F078A5
:05553F00A1F608F622B0
:103582009001E7E070107BFF7A0F79B612920090FB
:1035920001E77401F0229001E7E0640170599000A4
:1035A20000E06003023A17A249924E9001E8E090CF
:1035B20001B2F09001E9E09001B3F0900063E09075
:1035C20001B4F012869E9001B5EFF0128232D23F22
:1035D200126F36900094E0900006F0900096E09012
:1035E200000EF09000C0E09001FCF09001EE740734
:1035F200F09001E702374A9001E7E06402702C1272
:103602009575787DE66003023A17305803023A173F
:103612007628D2589001EEE014F0E06003023A17E7
:103622007402F09001E704F0C24A229001E7E064DC
:103632000360030237A8129575126D3BEF60781292
:1036420078A37BFF7A0F79B61292009000C0E070E7
:1036520003023700128F71EF64017057304A54C26F
:103662004A900050E0FFC39415504874DA2FF58257
:10367200E43400F583E0FFA248E4336F7035126E44
:103682009490004FE0641F602A9001E8E0FF9000F0
:1036920050E0B5071E9001E9E0FF900051E0B50748
:1036A200129000C0E09001FCF0C24A900094E090B9
:1036B2000006F0C24A80089000C0E09001FCF020B1
:1036C2005E0B9000C0E070051278A380319000C0BC
:1036D200E0600B9001FCE070051278A3802090025C
:1036E20044E0B4010A1278A3E4900244F0800F90FF
:1036F2000096E0601090000EE0700A1278A390012C
:10370200E77404F022787DE66003023A173058032A
:10371200023A179001EEE07033A249924E9001E80E
:10372200E09001B2F09001E9E09001B3F090006303
:10373200E09001B4F012869E9001B5EFF012823251
:10374200D23F126F369001EE7402F022127EA1EF88
:103752006401704F9001B0E0FF249AF582E43401D5
:10376200F583E09001B2F074852FF582E43401F51F
:1037720083E09001B3F09001B0E09001B4F01285C3
:10378200179001B5EFF09001B2E024DAF582E4344B
:1037920000F583E024FF924E128232D23F126F363E
:1037A20002385B02385B9001E7E0B4042C2062200F
:1037B20090021DE4F0A374FFF09002197401F0D29C
:1037C200621278A3E49001EFF09001E77405F02211
:1037D2007BFF7A0F79C70239FD9001E7E06405703B
:1037E20046787DE66003023A17305803023A17A280
:1037F20049924E9001E8E09001B2F09001E9E09028
:1038020001B3F09001B4741FF012962E9001B5EF3F
:10381200F01282321278A39001EE7403F0126F3626
:103822009001E77406F0229001E7E0FF6406703031
:10383200787DE66003023A17305803023A17900186
:10384200EEE0700F900095E0900001F09001E774B7
:1038520007F022787D7628D2589001EEE014F0220B
:10386200EF640760030239C2900001E0701312781E
:10387200919000BCE060031278B59001E77408F003
:1038820022128F71EF64016003023968900095E0A3
:10389200900001F0204A03023968C24A128F71EF88
:1038A200640160030239689001E8E0FF900050E093
:1038B200FEB50712900051E0FF9001E9E0B507065E
:1038C200E49001ECF022EEC39415400302396890B3
:1038D2000050E0FF24DAF582E43400F583E0FEA232
:1038E20048E4336E60030239689001ECE0FE701B1D
:1038F200A24892499001EBEFF0900051E09001EC68
:10390200F090004FE09001EDF0805B900050E0FFFE
:103912006E7053A24892499001E8EFF0900051E096
:103922009001E9F090004FE09001EAF0641F6036E8
:103932009001E8E0FFC39415502C74DA2FF582E46D
:103942003400F583E0FFA249E433B507199001E89A
:10395200E0FF9001E9E0FD7C001282CD9001E67467
:1039620002F0E40239F2787DE67055205852127F57
:103972006FEF6401704A9001B0E0FF249AF582E48F
:103982003401F583E09001B2F074852FF582E434BE
:1039920001F583E09001B3F09001B0E09001B4F042
:1039A2001285179001B5EFF09001B2E024DAF582AA
:1039B200E43400F583E024FF924E128232126F3615
:1039C2009001E7E06408703620622A90021D7418A4
:1039D200F0A3E4F090021904F0D2629001FBF0909F
:1039E20000A1E0FF78A1760008A607E49001E6F0C6
:1039F2009001E7F0227BFF7A0F79D802923590018D
:103A0200E7E0D39408400EE49001E6F09001E7F07D
:063A120078A1F608F6227F
:104E67009001E7E07076900063E090005AF09000C0
:104E77005B74FEF020625C9001F5E0FBB4010FE586
:104E8700402400FEE4341590021DF0A3CEF0EBB4ED
:104E970002119001F7E02400FEE4341690021DF0A1
:104EA700A3CEF09002197401F0D262900096E090C0
:104EB700000EF0900099E0900008F0900068E06024
:104EC7000BE49001E7F09001E60250449001E7748B
:104ED70001F0227BFF7A0F79E90251CC9001E7E0DC
:104EE7006401707B900000E060030251DEC26190B4
:104EF70001F5E064017025AF401294F5E54075F0C7
:104F070010A42483F9741135F0FA7BFF129200E59F
:104F17004075F010A42483F9741180359001F5E0F1
:104F2700640260030251DE9001F7E0FF12211D9039
:104F370001F7E075F010A424C3F9741435F0FA7B77
:104F4700FF1292009001F7E075F010A424C3F974E2
:104F57001435F0FA7BFF1292359001E702518A90DF
:104F670001E7E0640270591268F8EF602A206127B0
:104F77001278A39000A7E07002803E7BFF7A0F793A
:104F8700FA1292359000A7E0900009F0D2619000E4
:104F970065E0700312962530610A120086500512EB
:104FA70078A38015900096E070030251DE90000E02
:104FB700E060030251DE1278A39001E77403F02248
:104FC7009001E7E0B4032920621D90021DE4F0A3DD
:104FD70074FFF09002197401F0D262E49001F6F0C8
:104FE7009001E77404F0227BFF7A10790B0251CC11
:104FF7009001E7E0B4042D9000A8E060197BFF7AE8
:1050070010791C1292359000A8E0900002F09001F0
:10501700E77405F0800E900095E0900001F0900194
:10502700E77406F09001E7E0FFB40515900002E091
:10503700700F900095E0900001F09001E77406F082
:1050470022EF64066003025191900001E07015128F
:1050570078919000BCE060031278B5C2399001E7FF
:105067007407F022205D03025119900095E090002B
:1050770001F0303B46C23B9001F5E0B40109E54041
:10508700653F70030251DE9001F3E53FF0E075F0F4
:1050970010A42483F9741135F0FA7BFF1292009063
:1050A70001F3E0FF12889F900066E0600E9001F523
:1050B7007401F09001F3E0F540804B304154C24158
:1050C7009001F5E0B4020B9001F7E065357003023B
:1050D70051DE9001F4E535F0E075F010A424C3F932
:1050E700741435F0FA7BFF1292009001F4E0FF127E
:1050F700859A900066E0601A9001F57402F09001BD
:10510700F4E09001F7F0E49001E7F09001E6740510
:10511700F022C23BC241128F71EF64017069304ABD
:1051270066129625C239C24A900050E0FFC3941513
:10513700505574DA2FF582E43400F583E0FFA24876
:10514700E4336F7042A2489249900050E09001E822
:10515700F0900051E09001E9F090004FE09001EAF3
:10516700F0126E949001EAE0641F601B9001E8E082
:10517700FF9001E9E0FD7C001282CDE49001E7F0A9
:105187009001E67402F022C24A229001E7E0640728
:10519700703620622A90021D7418F0A3E4F0900282
:1051A7001904F0D2629001FBF09000A1E0FF78A112
:1051B700760008A607E49001E6F09001E7F0227B6D
:1051C700FF7A10792D0292359001E7E0D3940740DA
:0851D70006E4F09001E6F0226D
:105878009001E7E070127BFF7A10793E1292009057
:1058880001E77401F002789D9001E7E0640170621D
:10589800900000E06003025BA8C261900096E0906F
:1058A800000EF09000C0E09001FCF09001F5E0B42B
:1058B8000112AF401294F5E54075F010A42483F965
:1058C800741180209001F5E064026003025BA890E7
:1058D80001F7E0FF12211D9001F7E075F010A424F4
:1058E800C3F9741435F0FA7BFF1292359001E70280
:1058F8005B659001E7E0640260030259A3129575A5
:105908001268F8EF6033206130D2611278A39000FA
:10591800A7E0700B1278A39000C0E0701C80757B24
:10592800FF7A10794F1292359000A7E0900009F0A5
:10593800900065E07003129625306135120086509C
:10594800147BFF7A1079601292359000C0E0700DD8
:105958001278A3803F9000C0E09001FCF0128030E4
:105968009000C0E0600B9001FCE070051278A38005
:1059780023900244E0B40107E4F01278A380159064
:105988000096E07003025BA890000EE06003025BE3
:10599800A81278A39001E77403F0229001E7E0B41D
:1059A800032420621890021DE4F0A374FFF0900213
:1059B800197401F0D2629001E77404F0227BFF7A37
:1059C8001079710292359001E7E06404702512960F
:1059D80025E49001F6F09000A8E060307BFF7A1093
:1059E800791C1292359000A8E0900002F09001E72F
:1059F800025AF09001E7E0FFB40518900002E06059
:105A080003025BA8900095E0900001F09001E77414
:105A180006F022EF64066003025B6C900001E07000
:105A2800151278919000BCE060031278B5C23990E5
:105A380001E77407F022205D03025AF4900095E014
:105A4800900001F0303B4EC23B9001F5E0B40109F3
:105A5800E540653F7003025BA89001F3E53FF0E085
:105A680075F010A42483F9741135F0FA7BFF1292B3
:105A7800009001F3E0FF12889F900066E0601690A6
:105A880001F57401F09001F3E0F540E49001E7F0CE
:105A98009001E68053304154C2419001F5E0B402D0
:105AA8000B9001F7E065357003025BA89001F4E5FF
:105AB80035F0E075F010A424C3F9741435F0FA7BBE
:105AC800FF1292009001F4E0FF12859A900066E0C0
:105AD800601A9001F57402F09001F4E09001F7F07B
:105AE800E49001E7F09001E67405F022C23BC24160
:105AF800128F71EF64017069304A66129625C239B7
:105B0800C24A900050E0FFC39415505574DA2FF53F
:105B180082E43400F583E0FFA248E4336F7042A2C8
:105B2800489249900050E09001E8F0900051E090D0
:105B380001E9F090004FE09001EAF0126E949001B4
:105B4800EAE0641F601B9001E8E0FF9001E9E0FDD6
:105B58007C001282CDE49001E7F09001E67402F037
:105B680022C24A229001E7E0B4072620621A900276
:105B78001D7418F0A3E4F090021904F0D262E490C6
:105B880001E6F09001E7F0227BFF7A107982129209
:105B9800359001E7E0D394074006E4F09001E6F081
:015BA80022DA
:103A18009001E7E0702220621690021D7419F0A34D
:103A28007403F09002197401F0D2629001E7F07B00
:103A3800FF7A107993023E989001E7E0B401267B63
:103A4800FF7A1079A412920090005AE024DAF582E5
:103A5800E43400F583E024FF9249E4900241F090B9
:103A680001E7023E579001E7E06402704C900000C5
:103A7800E06003023EAAA249924E9001E8E090015C
:103A8800B2F09001E9E09001B3F0900063E090019A
:103A9800B4F012869E9001B5EFF0128232D23F1236
:103AA8006F3690008AE09001FDF0900096E090005B
:103AB8000EF09001E77403F0229001E7E0640360E0
:103AC80003023C1B129575126D3BEF606F1278A3D1
:103AD8007BFF7A1079A4129200128F71EF64017043
:103AE80057304A54C24A900050E0FFC394155048DA
:103AF80074DA2FF582E43400F583E0FFA248E4335A
:103B08006F7035126E9490004FE0641F602A900128
:103B1800E8E0FF900050E0B5071E9001E9E0FF9053
:103B28000051E0B5071290008AE09001FDF0C24A0A
:103B3800900094E0900006F0C24A800890008AE065
:103B48009001FDF0900244E0B40104E4F0801A9082
:103B580001FDE0700890008AE06002800C900096F9
:103B6800E0601090000EE0700A127BA49001E774E8
:103B780004F022787DE66003023EAA305803023E34
:103B8800AA9001EEE07032A249924E9001E8E090CE
:103B980001B2F09001E9E09001B3F0900063E09089
:103BA80001B4F012869E9001B5EFF0128232D23F36
:103BB800126F369001EE023E57127EA1EF6401703B
:103BC8004F9001B0E0FF249AF582E43401F583E0D8
:103BD8009001B2F074852FF582E43401F583E0900A
:103BE80001B3F09001B0E09001B4F0128517900194
:103BF800B5EFF09001B2E024DAF582E43400F58301
:103C0800E024FF924E128232D23F126F36023CCB32
:103C1800023CCB9001E7E0B4042620621A90021D12
:103C2800E4F0A374FFF09002197401F0D2629001DD
:103C3800E77405F01278A37BFF7A1079B5023E98F5
:103C48009001E7E064057049127BB31278A3787D90
:103C5800E66003023EAA305803023EAAA249924EE9
:103C68009001E8E09001B2F09001E9E09001B3F032
:103C78009001B4741FF012962E9001B5EFF01282E5
:103C8800329001EE7403F0126F369001E77406F07B
:103C9800229001E7E0FF64067030787DE660030259
:103CA8003EAA305803023EAA9001EEE0700F900041
:103CB80095E0900001F09001E77407F022787D7696
:103CC80028D2589001EEE014F022EF640760030256
:103CD8003E5E900001E070131278919000BCE060A5
:103CE800031278B59001E77408F022128F71EF641F
:103CF800017074900095E0900001F0303B2DC23BBC
:103D08009001F57401F0853F40C239E54075F01027
:103D1800A42483F9741135F0FA7BFF129200AF40A6
:103D280012889F900066E060028030304139C241BD
:103D38009001F7E535F075F010A424C3F974143533
:103D4800F0FA7BFF1292009001F7E0FF12859A903B
:103D580001F57402F0900066E0600CE49001E7F071
:103D68009001E67405F022C23BC241128F71EF64E4
:103D7800016003023E5B900095E0900001F0204A4C
:103D880003023E5B129625C239C24A9001E8E0FF61
:103D9800900050E0FEB50712900051E0FF9001E955
:103DA800E0B50706E49001ECF022EEC39415400359
:103DB800023E5B900050E0FF24DAF582E43400F51F
:103DC80083E0FEA248E4336E6003023E5B9001ECA0
:103DD800E0FE701BA24892499001EBEFF090005171
:103DE800E09001ECF090004FE09001EDF0806490DD
:103DF8000050E0FF6E705CA24892499001E8EFF035
:103E0800900051E09001E9F090004FE09001EAF055
:103E1800126E949001EAE0641F60389001E8E0FFB8
:103E2800C39415502E74DA2FF582E43400F583E03C
:103E3800FFA249E433B5071B9001E8E0FF9001E9D0
:103E4800E0FD7C001282CDE49001E7F09001E67479
:103E580002F022C24A229001E7E06408703520622D
:103E68002990021D7418F0A3E4F090021904F0D20E
:103E7800629001FBF09000A1E0FF78A1760008A60F
:103E880007E49001E6F09001E7F07BFF7A1079C62D
:103E98000292359001E7E0D394084006E4F09001DF
:033EA800E6F0221F
:104730009001E7E07046900063E090005AF090002E
:104740005B74FEF020622C900241E0FFB4010A90FD
:10475000021D7419F0A37401F0EFB4020A90021D57
:104760007419F0A37402F09002197401F0D26290EF
:1047700001E7F07BFF7A1079D71292359001E7E0DC
:1047800064017055900241E0B4011D900243E0F5D0
:10479000407BFF7A1079E8129200900243E0FF120A
:1047A000889F9001F57401F0900241E0B4021F90DF
:1047B0000243E09001F7F07BFF7A1079FB12920040
:1047C000900243E0FF12859A9001F57402F0E490A4
:1047D0000241F09001E7024A8F9001E7E064027025
:1047E0006C305D0512789D80031278A3900000E084
:1047F0006003024AE290008AE09001FDF09000968A
:10480000E090000EF09001F5E0B40112AF40129478
:10481000F5E54075F010A42483F97411802090010F
:10482000F5E064026003024AE29001F7E0FF122122
:104830001D9001F7E075F010A424C3F9741435F04D
:10484000FA7BFF1292359001E77403F0229001E7A2
:10485000E06403707C129575305D3C9001F5E0B426
:104860000115303B12E540B53F0D90008AE0900104
:10487000FDF0C23B12789D9001F5E0B4022030417A
:104880001D9001F7E0B5351690008AE09001FDF02B
:10489000C24112789D80071278A3C23BC2419002A8
:1048A00044E0B4010280209001FDE0700890008A8D
:1048B000E060028012900096E07003024AE29000ED
:1048C0000EE06003024AE2127BA49001E77404F058
:1048D000229001E7E0B4042320621790021DE4F067
:1048E000A374FFF09002197401F0D2629001E70204
:1048F0004A1F7BFF7A11790C024AD09001E7E064ED
:104900000570271278A31296259000A8E060307BEE
:10491000FF7A10791C1292359000A8E0900002F006
:104920001296259001E77406F0229001E7E0B406A4
:1049300015900002E0700F900095E0900001F0905B
:1049400001E77407F0229001E7E064076003024A80
:1049500096900001E070131278919000BCE0600323
:104960001278B59001E77408F022205D03024A2313
:10497000303B4EC23B9001F5E0B40109E540653F94
:104980007003024AE29001F3E53FF0E075F010A4F5
:104990002483F9741135F0FA7BFF1292009001F331
:1049A000E0FF12889F900066E060169001F57401A8
:1049B000F09001F3E0F540E49001E7F09001E6802B
:1049C0005E30415FC2419001F7E535F09001F5E0BE
:1049D000B4020B9001F7E065357003024AE29001E2
:1049E000F4E535F075F010A424C3F9741435F0FA29
:1049F0007BFF1292009001F4E0FF12859A9001F57E
:104A00007402F0900066E0601A9001F57402F09074
:104A100001F4E09001F7F0E49001E7F09001E67412
:104A200005F022C23BC241305D69304A66129625CC
:104A3000C239C24A900050E0FFC39415505574DA51
:104A40002FF582E43400F583E0FFA248E4336F7071
:104A500042A2489249900050E09001E8F090005145
:104A6000E09001E9F090004FE09001EAF0126E94BE
:104A70009001EAE0641F601B9001E8E0FF9001E90B
:104A8000E0FD7C001282CDE49001E7F09001E67435
:104A900002F022C24A229001E7E0640870352062E9
:104AA0002990021D7418F0A3E4F090021904F0D2CA
:104AB000629001FBF09000A1E0FF78A1760008A6CB
:104AC00007E49001E6F09001E7F07BFF7A11791D91
:104AD0000292359001E7E0D394084006E4F090019B
:034AE000E6F022DB
:105BA9009001E7E0FF703620623390021D7418F00F
:105BB900A37401F0900219F0D2629000BDE0FE6476
:105BC900016004EEB402079001E77401F022EE646B
:105BD900036004EEB404069001E7025D80EF6401FE
:105BE9006003025CD8128F71BF010890009BE0909E
:105BF9000005F0900005E0700F1278919000BCE06C
:105C090060031278B5025D039000BDE0B401097B21
:105C1900FF7A11792E025D2312788B9000BCE06027
:105C2900031278AF7BFF7A11793F129200787DE6F3
:105C39006003025E18305803025E189001EEE070AE
:105C490034D23F9000A2E024FF924E900063E0FF1F
:105C59009001B2F09000A0E09001B3F09001B4EF90
:105C6900F012869E9001B5EFF0128232126F3690D3
:105C790001EE025D80127EA1EF6401704FD23F9068
:105C890001B0E0FF249AF582E43401F583E0900144
:105C9900B2F074852FF582E43401F583E09001B305
:105CA900F09001B0E09001B4F01285179001B5EFC2
:105CB900F09001B2E024DAF582E43400F583E024BF
:105CC900FF924E128232126F36025DDA025DDA906D
:105CD90001E7E064026003025DE1129355BF010828
:105CE90090009BE0900005F0900005E0701F12788D
:105CF900919000BCE060031278B59000A1E0FF78B4
:105D0900A1760008A6079001E77403F0229000BD70
:105D1900E0B403097BFF7A11795002920012788B63
:105D29009000BCE060031278AF7BFF7A11796112B1
:105D39009200787DE66003025E18305803025E180F
:105D49009001EEE07035D23F9000A2E024FF924E20
:105D5900900063E0FF9001B2F09000A0E09001B3E1
:105D6900F09001B4EFF012869E9001B5EFF0128227
:105D790032126F369001EE7402F022127EA1EF64A6
:105D890001704ED23F9001B0E0FF249AF582E434CD
:105D990001F583E09001B2F074852FF582E43401B6
:105DA900F583E09001B3F09001B0E09001B4F012F6
:105DB90085179001B5EFF09001B2E024DAF582E49D
:105DC9003400F583E024FF924E128232126F36803E
:105DD900009001EEE014F0229001E7E0B4031E20E8
:105DE900621290021D7418F0A3E4F090021904F0F5
:105DF900D26280127BFF7A1179721292359001E793
:105E0900E0D394034009E49001E6F09001E7F02221
:0D008600900009E07002D322128030C322E6
:10803000205D030280D29001F5E064017040303B86
:108040003DC23BE540653F7035C261AF401294F5DB
:10805000E54075F010A42483F9741135F0FA7BFF24
:10806000129200E54075F010A42483F9741135F0E4
:10807000FA7BFF129235900099E0900008F0900191
:10808000F5E06402705A304157C2419001F8E5357D
:10809000F09001F7E0FF65357046C26112211D9036
:1080A00001F7E075F010A424C3F9741435F0FA7BDD
:1080B000FF1292009001F7E075F010A424C3F97448
:1080C0001435F0FA7BFF129235900099E090000889
:1080D000F022E47887F608F608F608F6C23BC241BB
:0180E000227D
:1000A600202020202020202020202020202020204A
:1000B6005245504541544552204E554D42455220D9
:1000C6002020202020202020203120746F20323054
:1000D600202053495445204E554D4245522020205C
:1000E6002020202020202020203120746F20393924
:1000F6008202001101021501148202011103041586
:1001060001632020202020202020202020202020C5
:1001160020202020202020202020202020202020D9
:10012600202020434F5552544553592042454550AF
:100136002020204354435353204F4E2048414E47DE
:10014600202020205553455220454E41424C452003
:10015600202020205245534552564520544F4E45A7
:10016600202020204E4554574F524B204D4F44459A
:100176002020204E4554574F524B204E554D424558
:100186005220202020202020202020202020202037
:100196002020202020202020202020202020202059
:1001A6002020202020202020202020202020202049
:1001B6002020202020202020202020202020202039
:1001C6002020202020202020202020202020313DFB
:1001D600454E2020202020202020202020204D4F6A
:1001E6004445202020202020202020202020544F5D
:1001F6004E4564010011020C150001640200110352
:100206000C15000164040011040C150001640800BB
:1002160011050C15000164100011060D150002C829
:10022600030111070A190101202020202020202087
:1002360020202020202020202020202020202020B8
:10024600202020202020202020434F555254455363
:100256005920424545502020204354435353204FB4
:100266004E2048414E4720202020555345522045D8
:100276004E41424C4520202020205245534552569F
:100286004520544F4E45202020204E4554574F526E
:100296004B204D4F44452020204E4554574F524B3E
:1002A600204E554D4245522020202020202020203F
:1002B6002020202020202020202020202020202038
:1002C6002020202020202020202020202020202028
:1002D6002020202020202020202020202020202018
:1002E6002020202020202020202020202020202008
:1002F60020202020313D454E202020202020202077
:10030600202020204D4F4445202020202020202042
:1003160020202020544F4E4564010011020C150088
:100326000164020011030C15000164040011040CA1
:1003360015000164080011050C1500016410001178
:10034600060D150001C8030111070A190101202035
:100356002020202020202020202020202020202097
:100366002020202020202020202020202020204364
:100376004F55525445535920424545502020202080
:100386005553455220454E41424C4520202020439E
:10039600524F535320544F4E45204D4F4445204312
:1003A600544353532F4443532043524F5353202017
:1003B6004E4554574F524B204D4F44452020204E1A
:1003C6004554574F524B204E554D42455220202002
:1003D6002020202020202020202020202020202017
:1003E60020202020202020202020313D454E202086
:1003F600202020202020202020204D4F4445202052
:1004060020202020202020202020544F4E45202030
:1004160020202020202020202020202020206401B1
:1004260000110209150001640200110309150001FB
:1004360064040011060A150001C8030111070C190E
:1004460001012020202020202020202020202020E4
:100456002020202020202020202020202020202096
:10046600202001010101010101010100000000003D
:100476000000000000000000000000000000000076
:100486000000000000000000000000000000000066
:100496000000000000000000000000000000000056
:1004A6000000000000000000000000000000000046
:1004B60000000000000000000000000020202020B6
:1004C6002020202020202020202020202020202026
:1004D6002020202020202020202020200101010192
:1004E6000101010101000000000000000000000001
:1004F60000000000000000000000000000000000F6
:1005060000000000000000000000000000000000E5
:1005160000000000000000000000000000000000D5
:1005260000000000000000000000000000000000C5
:100536000000000000002020202020202020202075
:1005460020202020202020202020202020202020A5
:1005560020202020202001010101010101010120AC
:100566002020202020202020202020202020202085
:100576002020202020202020202020202020202075
:1005860054454C434F2050524F4752414D20202056
:10059600524144494F2050524F4752414D2020204E
:1005A60050484F4E452050524F4752414D20202033
:1005B600434F4D50552050524F4752414D20202019
:1005C6002041434345535320434F44452020204474
:1005D600544D462054454C434F204C4556454C44BB
:1005E600544D4620524144494F204C4556454C42B5
:1005F60045455020524144494F204C4556454C42B2
:100606004545502054454C434F204C4556454C4398
:1006160057494420524144494F204C4556454C5673
:100626004F49434520524144494F204C45564C566C
:100636004F4943452054454C434F204C45564C505A
:1006460041474520524144494F204C4556454C436D
:100656005443535320524144494F204C45564C4431
:10066600435320524144494F204C4556454C204C5B
:10067600545220524144494F204C4556454C205235
:10068600505420524144494F204C4556454C205425
:10069600454C434F20524144494F204C45564C52FD
:1006A6004144494F2054454C434F204C45564C52EB
:1006B6004144494F204C494D4954204C45564C2005
:1006C600434F53204F5220535155454C4348202009
:1006D60020434F5320504F4C4152495459202043F8
:1006E6004F53205452494747455220564F4C544386
:1006F6004F5320414351554953542054494D454386
:100706004F532052454C454153452054494D4520B1
:1007160053454E534520504F4C415249545920534E
:10072600454E205452494747455220564F4C545344
:10073600454E20414351554953542054494D455344
:10074600454E2052454C454153452054494D452080
:100756004C545220484F4C442044454C415920505B
:100766005454205455524E4F46462054494D4552F6
:10077600455045415445522054494D454F55542006
:1007860020414E54492D4B45524348554E4B20204F
:1007960020535155454C4348205441494C20202074
:1007A60043544353532F44435320484F4C44204310
:1007B600524F535320425553592044454C415943B7
:1007C600524F5353204255535920484F4C442020F2
:1007D600204C54522053594E432042495420202045
:1007E600414456414E43454420204C4F434B202024
:1007F60020202020202020202020202020202020F3
:1008060020202020202020202020202020202020E2
:1008160020202020202020202020202020202020D2
:1008260020202020202020202020202020202020C2
:100836002020202020202020202020313D454E2031
:1008460020202020202020202020524154494F20C3
:1008560020202020202020202020303D434F5320E0
:1008660020202020202020202020313D504F5320C2
:10087600202020202020202020202031204D532001
:10088600202020202020202020203130204D5320E1
:10089600202020202020202020313030204D5320C1
:1008A60020202020202020202020202053454320C7
:1008B600202020202020202020313D534B4950204D
:1008C6002020202020202020202020202020202022
:1008D6002020202020202020202020202020202012
:1008E6005052494F52495459204C4556454C2020A8
:1008F6004C545220454E434F444520504F4C2020E7
:100906004C5452204445434F444520504F4C2020E0
:10091600205445535420494420434F444520204900
:10092600444C45204D45535341474520544D522094
:100936002020204152454120424954202020202099
:100946004D4153544552204F5220534C4156452059
:1009560044435320454E434F444520504F4C20209E
:10096600444353204445434F444520504F4C202098
:10097600434F5552544553592044454C4159202024
:10098600202048414E472054494D452020202043F1
:100996004152524945522044524F5020444C59200E
:1009A600204143434553532044454C41592020534D
:1009B600544154494F4E204944204D4F4445202030
:1009C600564F494345204F52204357494420202043
:1009D60020494420494E54455256414C202020205F
:1009E6002020435749442053504545442020202089
:1009F60043574944204652455155454E43592020B8
:100A06002043574944204D45535341474520202014
:100A16005455524E5F4F4E2044454C41592020209C
:100A26005455524E5F4F46462044454C415920206E
:100A360042454550204652455155454E4359205250
:100A4600455045415445522044495341424C452066
:100A56004155582052454C4159204D4F4445202080
:100A660043524F53532042555359204D4F4445202E
:100A76005245504541544552204741494E20202079
:100A86002054454C434F204741494E202020204EBC
:100A96004554574F524B2048414E4754494D4520E7
:100AA6002020202020202020204C4556454C202068
:100AB600202020202020202020303D4E4F524D2047
:100AC6002020202020202020202020434F44452085
:100AD6002020202020202020202020415245412077
:100AE60020202020202020303D4D415354455220C7
:100AF600202020202020202020202031204D53207F
:100B0600202020202020202020203130204D53205E
:100B1600202020202020202020313030204D53203E
:100B26002020202020202020203130205345432023
:100B36002020202020202020202031204D494E201A
:100B460020202020202020202020204D4F444520FA
:100B56002020202020202020303D564F494345208C
:100B660020202020202020202020204652455120D1
:100B76002020202020202020202020313D454E20EE
:100B860020414C41524D20434F554E5420202020A9
:100B9600524553544F524520434F554E5420202022
:100BA6002020494E54455256414C202020202020DA
:100BB6004E4554574F524B20434F44452020204921
:100BC6004E544552434F4E4E454354204D4F444E8E
:100BD6004554574F524B20494E414354495645823E
:100BE600010011022D15000182010111032D1500CE
:100BF6000182010211042D15000182010311052D48
:100C060015000178060411060119010182030A1173
:100C1600072E1500FF82030B11082E1500FF820315
:100C26000C11092E1500FF82030D110A2E1500FF67
:100C360082030E110B2E1500FF82030F110C2E15C9
:100C460000FF820310110D2E1500FF820311110EF5
:100C56002E1500FF820312110F2E1500FF820313BB
:100C660011102E1500FF82031411112E1500FF829C
:100C7600031511122E1500FF82031611132E1500EF
:100C8600FF82031711142E1500FF82031811152E6B
:100C96001500FF82011911162F15000182011A1184
:100CA600173015000182031B11182E1500FF820252
:100CB6001C11193115006382021D111A32150063C9
:100CC60082011E111B3015000182031F111C2E15F7
:100CD60000FF820220111D31150063820221111EC0
:100CE60032150063820222111F3315026382032329
:100CF6001120321501FF8203241121341502FF82CF
:100D060002251122331500638202261123321500B3
:100D160063820227112433150363820228112532C8
:100D26001500638203291126331500FA82012A1160
:100D3600273515000182012B11385415010982014E
:100D46002C11395515000182012D113A5515000156
:100D560082032E113B561501FA82032F113C5C15B6
:100D660000FF820130113D57150001820131113E0D
:100D760058150001820132113F55160001820133D8
:100D860011405515000182023411415A1500638243
:100D9600023511425B15006382023611435A150073
:100DA6006382023711445A15006382013811455E89
:100DB60015000182013911465F15000182023A11C0
:100DC600475D15006382023B114859150463820290
:100DD6003C114960150114BE0A3D114A5611000026
:100DE600820247114B5A150063820248114D601565
:100DF6000114820149114E5E15000282014A114F0B
:100E06006115000182014B11505E15000482014CF0
:100E160011515415010982014D11525415010982CF
:100E2600024E11533415006382014F116201150001
:100E36000982015011630115000982025111645D96
:100E4600150163C803521165011501018201541190
:100E5600665E1500028203551167341500FF010115
:100E66000200000200000200000000000001010173
:100E76003132333435361432320532FFFFFF191959
:100E8600196464C8FF000180000A0180000A1E1A66
:100E9600B400001E1E1E0001000002010001000039
:100EA6000A1E630A000100050520202020202020BC
:100EB6002020200A050000000101140000010000A6
:020EC60000002A
:109200008B708A7189727F01127B8AE490013FF032
:1092100090013FE0FFC39410501AAB70AA71A9727D
:109220008F827583001281A5FF127B5B90013FE066
:0592300004F080DC22C7
:10677A008B708A71897290024BE0B4110040030257
:10678A0068F7906793F82828730267C60267CE02F3
:10679A0067DE0267F102680402681702682A026863
:1067AA003D02685002686302687502688702689948
:1067BA000268AB0268BD0268CF0268E17F01127B02
:1067CA008A0268F1AB70AA71A97212818CFF127BDE
:1067DA005B0268F1AB70AA71A9729000011281A5DF
:1067EA00FF127B5B0268F1AB70AA71A9729000027A
:1067FA001281A5FF127B5B0268F1AB70AA71A972C4
:10680A009000031281A5FF127B5B0268F1AB70AAAC
:10681A0071A9729000041281A5FF127B5B0268F1D4
:10682A00AB70AA71A9729000051281A5FF127B5B59
:10683A000268F1AB70AA71A9729000061281A5FFD5
:10684A00127B5B0268F1AB70AA71A9729000071201
:10685A0081A5FF127B5B0268F1AB70AA71A97290E5
:10686A0000081281A5FF127B5B807CAB70AA71A91C
:10687A00729000091281A5FF127B5B806AAB70AA35
:10688A0071A97290000A1281A5FF127B5B8058AB36
:10689A0070AA71A97290000B1281A5FF127B5B800E
:1068AA0046AB70AA71A97290000C1281A5FF127BE7
:1068BA005B8034AB70AA71A97290000D1281A5FF9A
:1068CA00127B5B8022AB70AA71A97290000E1281B2
:1068DA00A5FF127B5B8010AB70AA71A97290000FA2
:0E68EA001281A5FF127B5B90024BE004F022AE
:109235008B708A7189727F11127B8AE490013FF0ED
:1092450090013FE0FFC39410501AAB70AA71A97248
:109255008F827583001281A5FF127B5B90013FE031
:0592650004F080DC2292
:10431F00E4900203F0A3F0900205F0900143F0A3A4
:10432F00F0900144E02400F582E43404F583E4F0D6
:10433F00900144E004F07006900143E004F0900116
:10434F0043E07004A3E0648070D7E490013FF090E5
:10435F00013FE0FFC3940240030243F0EF900E646D
:10436F0093FF900205E0FE04F074002EF582E43412
:10437F0004F583EFF0900205E06480705B90020318
:10438F00E0FEA3E07807C333CE33CED8F9FF7C0429
:10439F007D00127314E4900143F0A3F0900144E008
:1043AF002400F582E43404F583E4F0900144E00442
:1043BF00F07006900143E004F0900143E07004A315
:1043CF00E0648070D7E4900205F0900204E004F0FE
:1043DF007006900203E004F090013FE004F0024306
:1043EF005EE4900142F0E4900140F0A3F0E490010C
:1043FF003FF090013FE0FFC394034003024493EF6B
:10440F00900E6693FF900205E0FE04F074002EF507
:10441F0082E43404F583EFF0900205E06480705B72
:10442F00900203E0FEA3E07807C333CE33CED8F972
:10443F00FF7C047D00127314E4900143F0A3F0900D
:10444F000144E02400F582E43404F583E4F09001A4
:10445F0044E004F07006900143E004F0900143E063
:10446F007004A3E0648070D7E4900205F09002041A
:10447F00E004F07006900203E004F090013FE004C6
:10448F00F0024401900141E004F07006900140E019
:10449F0004F0C3900141E09433900140E094005048
:1044AF00030243FC900142E004F0E0C39414500374
:1044BF000243F5E4900142F0E4900140F0A3F0E4F0
:1044CF0090013FF090013FE0FFC39403400302458A
:1044DF0065EF900E6993FF900205E0FE04F0740003
:1044EF002EF582E43404F583EFF0900205E064804A
:1044FF00705B900203E0FEA3E07807C333CE33CEA8
:10450F00D8F9FF7C047D00127314E4900143F0A3EB
:10451F00F0900144E02400F582E43404F583E4F0E4
:10452F00900144E004F07006900143E004F0900124
:10453F0043E07004A3E0648070D7E4900205F0902C
:10454F000204E004F07006900203E004F090013FD3
:10455F00E004F00244D3900141E004F070069001B2
:10456F0040E004F0C3900141E09470900140E0946A
:10457F000050030244CE900142E004F0E0C39414D3
:10458F0050030244C7E4900140F0A3F0E490013FD0
:10459F00F090013FE0FFC394034003024632EF90D7
:1045AF000E6C93FF900205E0FE04F074002EF5826E
:1045BF00E43404F583EFF0900205E06480705B90C3
:1045CF000203E0FEA3E07807C333CE33CED8F9FF62
:1045DF007C047D00127314E4900143F0A3F090016A
:1045EF0044E02400F582E43404F583E4F0900144C0
:1045FF00E004F07006900143E004F0900143E07096
:10460F0004A3E0648070D7E4900205F0900204E008
:10461F0004F07006900203E004F090013FE004F014
:10462F000245A0900141E004F07006900140E004C3
:10463F00F0C3900141E09488900140E0941350033F
:10464F0002459B8000E4900140F0A3F0E490013F0D
:10465F00F090013FE0FFC3945640030246F2EF9003
:10466F000E7293FF900205E0FE04F074002EF582A7
:10467F00E43404F583EFF0900205E06480705B9002
:10468F000203E0FEA3E07807C333CE33CED8F9FFA1
:10469F007C047D00127314E4900143F0A3F09001A9
:1046AF0044E02400F582E43404F583E4F0900144FF
:1046BF00E004F07006900143E004F0900143E070D5
:1046CF0004A3E0648070D7E4900205F0900204E048
:1046DF0004F07006900203E004F090013FE004F054
:1046EF00024660900141E004F07006900140E00442
:1046FF00F0C3900141E09414900140E09400500306
:10470F0002465B900203E0FEA3E07807C333CE338B
:10471F00CED8F9FF7C047D00127314127BA4027BA8
:01472F00B3D6
:1095D900E4900061F0A3F0FFFE1272BD900063EF0A
:0295E900F0226E
:10836300755401755500755672E4900249F0A3F0F7
:10837300900249E0FAA3E0FBC39456EA940050400C
:10838300900063E075F056A42478FFE5F03460CFE5
:108393002BCF3AFE900061F0A3EFF01272BDAB5405
:1083A3000556E556AA557002055514F9EF1281D208
:1083B30090024AE004F070B8900249E004F080B003
:1083C3009000A3E07004D2598002C25990009FE04C
:1083D30024FF925090009EE024FF92449000A5E079
:1083E30024FF924F9000A4E024FF9245900084E084
:0283F300F52E65
:0183F5002265
:108C56007554017555007556C7E4900249F0A3F0A6
:108C6600900249E0FEA3E0FFC39414EE9400503B4B
:108C76007C007D561281E4EF24F9FFEE3460FE900D
:108C86000061F0A3EFF01272BDAB540556E556AA8B
:108C9600557002055514F9EF1281D290024AE0048C
:0B8CA600F070BD900249E004F080B5C2
:018CB10022A0
:108CB2007554017555007556DBE4900249F0A3F036
:108CC200900249E0FEA3E0FFC39414EE9400503BEF
:108CD2007C007D561281E4EF24FEFFEE3460FE90AC
:108CE2000061F0A3EFF01272BDAB540556E556AA2F
:108CF200557002055514F9EF1281D290024AE00430
:0B8D0200F070BD900249E004F080B565
:018D0D002243
:10889F008F70E490013FF090013FE0FBC3940350D1
:1088AF003E900063E075F099A42469FDE5F034FF74
:1088BF00FCE57075F003A42DFFE5F03CFEEB7C00AA
:1088CF002FFFEC3EFE1272BD90013FE02469F5824E
:1088DF00E43400F583EFF090013FE004F080B890AE
:1088EF000069E0FE5401900064F0EE5402900065C0
:1088FF00F0900069E05404900066F0EE5408900088
:0D890F0067F0900069E05410900068F022BD
:10859A008F70E490013FF090013FE0FBC3940350D9
:1085AA0044900063E0FF7E007C017D501281E4EF7D
:1085BA0024A6FDEE340AFCE57075F003A42DFFE550
:1085CA00F03CFEEB7C002FFFEC3EFE1272BD9001E8
:1085DA003FE02469F582E43400F583EFF090013F2F
:1085EA00E004F080B2900069E0FE5401900064F06B
:1085FA00EE5402900065F0900069E0540490006621
:10860A00F0EE5408900067F0900069E05410900072
:03861A0068F022E3
:0682CD008F708C718D72B0
:1082D300E4900249F0A3F0E57224FFFFE57134FF57
:1082E300FE7C007D031281E4AA06AB07AE70E57045
:1082F30025E0CE75F0EEA4FFE5F02EFEEF2448FF57
:10830300EE3423CF2BCF3AFE90024AE02FFF9002A8
:1083130049E03EFE1272BD90024AE02469F582E410
:108323003400F583EFF090024AE004F07006900207
:1083330049E004F0C390024AE09403900249E094B8
:10834300004094900069E0FE540190006FF0EE54F9
:0F83530002900070F0900069E05404900071F007
:0183620022F8
:1094B6002020202020534C415645202020202020CB
:1094C60020202020204D415354455220202020208A
:0E960B00127AB8127BA4127BB37F01027B8A15
:1092FA00900003740AF0900003E070FA9000A3E073
:10930A007BFF60067A9479B680047A9479C61292C1
:0E931A0035900003740AF0900003E070FA2210
:10762C00C0D0C0E0C0F0C000A88475840FE55954E8
:10763C0007B4000D85E8F0A2F09220A2F19221800F
:10764C0076B4010D85E8F0A2F09222A2F19223808B
:10765C0066B4020D85E8F0A2F09224A2F192258086
:10766C0056B4030D85E8F0A2F09226A2F192278081
:10767C0046B4040D85E8F0A2F09218A2F19219809C
:10768C0036B4050D85E8F0A2F0921AA2F1921B8097
:10769C0026B4060D85E8F0A2F0921CA2F1921D8092
:1076AC001685E8F0A2F0921EA2F1921F7559FF8583
:1076BC00231E85241FD2650559755A0A8884D0006B
:1076CC00D0F0D0E0D0D03220640122D2B7E55B54A8
:1076DC0007B4000AA22F92F7A22E92F6805EB40194
:1076EC000AA22D92F7A22C92F68051B4020AA22B78
:1076FC0092F7A22A92F68044B4030AA22992F7A226
:10770C002892F68037B4040AA23792F7A23692F682
:10771C00802AB4050AA23592F7A23492F6801DB4E1
:10772C00060AA23392F7A23292F68010B40721A275
:10773C003192F7A23092F6C264755BFF055B7584DB
:10774C000F85E8E0A2F692E6A2F792E7F5E8C2B759
:01775C00220A
:105E1900202020445350205265736574202020208F
:105E29000000000000000004000000080000000C51
:105E39000000001000000014000000180000001C01
:105E49000000002000000024000000280000002CB1
:105E59000000003000000034000000380000003C61
:105E69000000004000000044000000480000004C11
:105E79000000005000000054000000580000005CC1
:105E89000000006000000064000000680000006C71
:105E99000000007000000074000000780000007C21
:105EA9000000108000001084000010880000108C91
:105EB9000000109000001094000010980000109C41
:105EC900000010A0000010A4000010A8000010ACF1
:105ED900000010B0000010B4000010B8000010BCA1
:105EE900000010C0000010C4000010C8000010CC51
:105EF900000010D0000010D4000010D8000010DC01
:105F0900000010E0000010E4000010E8000010ECB0
:105F1900000010F0000010F4000010F8000010FC60
:105F29000000218000002184000021880000218CCC
:105F39000000219000002194000021980000219C7C
:105F4900000021A0000021A4000021A8000021AC2C
:105F5900000021B0000021B4000021B8000021BCDC
:105F6900000021C0000021C4000021C8000021CC8C
:105F7900000021D0000021D4000021D8000021DC3C
:105F8900000021E0000021E4000021E8000021ECEC
:105F9900000021F0000021F4000021F8000021FC9C
:105FA9000000318000003184000031880000318C0C
:105FB9000000319000003194000031980000319CBC
:105FC900000031A0000031A4000031A8000031AC6C
:105FD900000031B0000031B4000031B8000031BC1C
:105FE900000031C0000031C4000031C8000031CCCC
:105FF900000031D0000031D4000031D8000031DC7C
:10600900000031E0000031E4000031E8000031EC2B
:10601900000031F0000031F4000031F8000031FCDB
:016029000076
:103EAB00900208E0FFEF707C90021AE0FFEFD394D2
:103EBB0003400302431E20650302431EC2659002AA
:103ECB0002741EF0900217E51EF0A3E51FF090029E
:103EDB0017E0FEA3E0FFEE541FFE900211EEF0A3DD
:103EEB00EFF0900217E0FEA3E0FFEEC4135407FFC0
:103EFB007E00900217EEF0A3EFF0900218E0FF9017
:103F0B00020AEFF0900209E4F0900217E0FEA3E042
:103F1B00FFEF4E7004D2632222900218E0FF900252
:103F2B0008EFF022900208E0FFEFB4011A206503BE
:103F3B0002431E900213E51EF0A3E51FF0C265D2EB
:103F4B0063900208E4F022900208E0FFEF64027035
:103F5B004320650302431EC265900209E0FFEF7028
:103F6B0011900213E51EF0A3E51FF0900209E00487
:103F7B00F022900209E0FFEFB40112900215E51E4A
:103F8B00F0A3E51FF0D263900208E4F02290020840
:103F9B00E4F02222900208E0FFEF6403600302408A
:103FAB00C120650302431E900201740AF0C26590A2
:103FBB000209E0FFEF7029900213E51EF0A3E51F45
:103FCB00F090020FE4F0A3E4F090020BE4F0A3E412
:103FDB00F090020DE4F0A3E4F0900209E004F0226B
:103FEB00900209E0FFEF64017079900217E51EF073
:103FFB00A3E51FF0900217E0FEA3E0FF90020CE098
:10400B002FF090020BE03EF0900217E0FCA3E0FDD6
:10401B0090020DE475F0011281F6AFF0FEEF25E092
:10402B00FFEE33FE74002FF58274043EF583ECF043
:10403B00A3EDF0900210E004F0700690020FE00484
:10404B00F0900211E0FEA3E0FF90020FE0FCA3E072
:10405B00FDED6F7002EC6E600302431E900209745B
:10406B0002F022900209E0FFEF6402704290021509
:10407B00E51EF0A3E51FF0900208E4F090020BE0C0
:10408B00FEA3E0FF900215E0FCA3E0FDEDB50717E2
:10409B00ECB50613900213E0FEA3E0FF1293827FB0
:1040AB00007E901295B4227F017E901295B42290DF
:1040BB000208E4F02222900208E0FFEF64046003A0
:1040CB000241F620650302431E900201740AF0C2FE
:1040DB0065900209E0FFEF7029900213E51EF0A333
:1040EB00E51FF090020FE4F0A3E4F090020BE4F074
:1040FB00A3E4F090020DE4F0A3E4F0900209E004D5
:10410B00F022900209E0FFEF64017073900217E553
:10411B001EF0A3E51FF0900217E0FEA3E0FF900254
:10412B000CE02FF090020BE03EF0900217E0FCA3A6
:10413B00E0FD90020DE475F0011281F6AFF0FEEF99
:10414B0025E0FFEE33FE74002FF58274043EF583F9
:10415B00ECF0A3EDF0900210E004F0700690020F6B
:10416B00E004F090020FE0FEA3E0FFEF64007003A9
:10417B00EE6402600302431E900209E004F02290F9
:10418B000209E0FFEF6402705B755C55900215E568
:10419B001EF0A3E51FF090020BE0FEA3E0FF9002E0
:1041AB0015E0FCA3E0FDEDB50727ECB50623900267
:1041BB0011E0FEA3E0FF127BC27F007E901295B44C
:1041CB00900213E0FEA3E0FFEF4E6012755DAA8034
:1041DB000D755C00755D007F017E901295B49002A9
:1041EB0008E4F022900208E4F02222900208E0FF9B
:1041FB00EF6405600302430920650302431E90022E
:10420B0001740AF0C265900209E0FFEF7029900279
:10421B0013E51EF0A3E51FF090020FE4F0A3E4F00A
:10422B0090020BE4F0A3E4F090020DE4F0A3E4F0B1
:10423B00900209E004F022900209E0FFEF640170A4
:10424B0076900217E51EF0A3E51FF0900217E0FE33
:10425B00A3E0FF90020CE02FF090020BE03EF090F9
:10426B000217E0FCA3E0FD90020DE475F001128152
:10427B00F6AFF0FEEF25E0FFEE33FE74002FF58274
:10428B0074043EF583ECF0A3EDF0900210E004F023
:10429B00700690020FE004F0900211E0FEA3E0FF25
:1042AB0090020FE0FCA3E0FDED6F7002EC6E70630B
:1042BB00900209E004F022900209E0FFEFB402370C
:1042CB00900215E51EF0A3E51FF0900208E4F090B4
:1042DB00020BE0FEA3E0FF900215E0FCA3E0FDED76
:1042EB00B5070CECB506087F007E901295B4227FC3
:1042FB00017E901295B422900208E4F022229002E3
:10430B0008E0FFEFD39405400A900208E4F0900216
:04431B0009E4F0229F
:102FF30090021AE0FFEF702A900208E0FFEFD394EB
:1030030002400302358130640302358120620302EA
:103013003581900219E0FF90021AEFF090021BE451
:10302300F02290021AE0FFEFB4011790021DE0FEB8
:10303300A3E0FFEE4420FE1295B4C26290021AE4AC
:10304300F02290021AE0FFEF6402705290021BE03C
:10305300FFEF701D30640302358190021DE0FEA373
:10306300E0FFEE4440FE1295B490021BE004F02210
:103073002290021BE0FFEFB4011E3064030235818E
:1030830090021FE0FEA3E0FF1295B4C26290021A01
:10309300E4F090021BE4F02290021AE4F022900282
:1030A3001AE0FFEF6403707290021BE0FFEF701CE5
:1030B30030640302358190021DE0FEA3E0FFEE447D
:1030C30060FE1295B490021BE004F02290021BE014
:1030D300FFEFB4011830640302358190021FE0FE54
:1030E300A3E0FF1295B490021BE004F02290021BB0
:1030F300E0FFEFB4021E306403023581900221E049
:10310300FEA3E0FF1295B4C26290021AE4F09002AB
:103113001BE4F02290021AE4F02290021AE0FFEF7F
:10312300640460030232BD90021BE0FFEF70339032
:10313300021DE0FEA3E0FF90021FE0FCA3E0FD12EE
:103143008DBD900225E4F0A3E4F0900227E4F0A300
:103153007480F0900223E4F0A3E4F090021BE004F7
:10316300F02290021BE0FFEFB4011C306403023530
:103173008190021DE0FEA3E0FFEE4480FE1295B4B1
:1031830090021BE004F02290021BE0FFEFB4021850
:1031930030640302358190021FE0FEA3E0FF129525
:1031A300B490021BE004F02290021BE0FFEF6403E3
:1031B3007063306403023581900223E475F00112D9
:1031C30081F6AFF0FEEF25E0FFEE33FE74002FF53E
:1031D3008274043EF583E0F56BA3E0F56CAF6CAE4F
:1031E3006B1295B4900226E0256CF0900225E03531
:1031F3006BF0900228E024FFF0900227E034FFF008
:10320300900227E0FEA3E0FFEF4E6002222290022D
:103213001BE004F02290021BE0FFEFB4041E3064B5
:1032230003023581900225E0FEA3E0FF1295B490DE
:10323300021C7464F090021BE004F02290021BE075
:10324300FFEF6405706E90021CE0FFEF70199002AF
:103253002AE004F07006900229E004F090021AE4D8
:10326300F090021BE4F022206503023581C26585DC
:103273001E6D851F6E90021BE4F0E56EB40011E530
:103283006DB4900C90021AE4F090021BE4F0C26259
:10329300E56E64017004E56D64906003023581900E
:1032A300021BE4F090022AE004F07006900229E089
:1032B30004F0222290021AE4F02290021AE0FFEFB7
:1032C3006405600302358190021BE0FFEF702B90D1
:1032D3000225E4F0A3E4F09002277402F0A3E4F0E3
:1032E300900223E4F0A3E4F090021DE0FEA3E0FFCC
:1032F30012882090021BE004F02290021BE0FFEFF3
:10330300B4011C30640302358190021DE0FEA3E08A
:10331300FFEE44A0FE1295B490021BE004F022904D
:10332300021BE0FFEF640270633064030235819097
:103333000223E475F0011281F6AFF0FEEF25E0FF02
:10334300EE33FE74002FF58274043EF583E0F56BD3
:10335300A3E0F56CAF6CAE6B1295B4900226E0253A
:103363006CF0900225E0356BF0900228E024FFF02A
:10337300900227E034FFF0900227E0FEA3E0FFEF86
:103383004E6002222290021BE004F02290021BE016
:10339300FFEFB4031E306403023581900225E0FE83
:1033A300A3E0FF1295B490021C7464F090021BE03A
:1033B30004F02290021BE0FFEF6404706B90021C88
:1033C300E0FFEF701490022AE004F07006900229E7
:1033D300E004F090021BE4F022306546C265851ECE
:1033E3006D851F6E90021BE4F0E56EB40011E56D70
:1033F300B4900C90021AE4F090021BE4F0C262E570
:103403006E64017004E56D6490600302358190027F
:103413002AE004F07006900229E004F090021BE415
:10342300F02290021AE4F02290021BE0FFEF7020DA
:10343300900225E4F0A3E4F09002277402F0A3E4E1
:10344300F0900223E4F0A3E4F090021BE004F022E6
:1034530090021BE0FFEFB4011C306403023581903E
:10346300021DE0FEA3E0FFEE44C0FE1295B49002FD
:103473001BE004F02290021BE0FFEF640270633054
:103483006403023581900223E475F0011281F6AFE3
:10349300F0FEEF25E0FFEE33FE74002FF582740497
:1034A3003EF583E0F56BA3E0F56CAF6CAE6B129564
:1034B300B4900226E0256CF0900225E0356BF09085
:1034C3000228E024FFF0900227E034FFF090022767
:1034D300E0FEA3E0FFEF4E6002222290021BE00415
:1034E300F02290021BE0FFEFB4031E3064030235A9
:1034F30081900225E0FEA3E0FF1295B490021BE049
:1035030004F090021C7464F02290021BE0FFEF644D
:1035130004706690021CE0FFEF701990022AE00429
:10352300F07006900229E004F090021BE4F0900290
:103533001AE4F022306547C265851E6D851F6E90C3
:10354300021BE4F0E56EB40011E56DB4900C90023B
:103553001AE4F090021BE4F0C262E56EB4011FE5C9
:103563006DB4901A90021BE4F090022AE004F0700C
:0E35730006900229E004F0222290021AE4F0F1
:013581002227
:047BC2008E0F8F1083
:107BC600D3E510947DE50F940040047F0180027F89
:107BD60000C3E510943FE50F940050047E01800237
:107BE6007E00EE4FFFEF6003027CBEE510AE0F781D
:107BF60002C333CE33CED8F9FF742C2FF582745ED0
:107C06003EF583E493F511740193F512E510AE0F7A
:107C16007802C333CE33CED8F9FF742A2FF5827497
:107C26005E3EF583E493FE740193FF8F179002087E
:107C3600E0FFEF6405FF900247EFF0900209E0FFD6
:107C4600EF6401FF900248EFF0AD12AC11AF1712CE
:107C5600906F900208E0FFEF6405FF900247EFF097
:107C6600900209E0FFEF6403FF900248EFF07515FC
:107C760000751600C3E51594045033AE15AF16749F
:107C8600002FF58274043EF583E0FF7E008E138F8D
:107C960014AB14AD12AC11AF17128EE90512E51232
:107CA600700205110516E5167002051580C69002CC
:087CB60047E4F0900248E4F0FD
:017CBE0022A3
:109382008E188F197B017A047900AC02AD01AF19F6
:10939200AE18127314E5192480FFE5183400FE7B21
:0D93A200017A047980AC02AD01127314222F
:048820008E5E8F5F7A
:10882400E55FAE5E7802C333CE33CED8F9FF742C45
:108834002FF582745E3EF583E493F560740193F53D
:1088440061E55FAE5E7802C333CE33CED8F9FF74F0
:108854002A2FF582745E3EF583E493FE740193FF40
:108864008F64756200756300C3E5629404502BAD98
:1088740061AC60AF64129496AC62AD6374002DF584
:108884008274043CF583EFF00561E56170020560D4
:0A8894000563E5637002056280CE03
:01889E0022B7
:088DBD008E658F668C678D68DE
:108DC500756900756A00E5662401FFE5653400FEF6
:108DD500EF25E0FFEE33FEC3E56A9FE5699E502966
:108DE5000568E568AE677002056714FF1272BDACD1
:108DF50069AD6A74002DF58274043CF583EFF005C6
:098E05006AE56A7002056980BD8E
:018E0E002241
:1095B4008E768F772064FD857625857726755B000A
:0395C400D264224C
:10713E0020630302727BC26390020AE0FFEF6003DA
:10714E0002720C900211E0FEA3E0FFEFB4FF22EEFC
:10715E00B41F1E7BFF7A5E791912920090000374A1
:10716E000AF0900003E0FFEF70F875840075EF03EE
:10717E0022900211E0FEA3E0FFEEFF7E008F7890DA
:10718E000212E0FFEF54FFF579E57870107FFF8F64
:10719E0079900241E4F09002447401F022E578B453
:1071AE001514E579C39433500D9002417401F0909B
:1071BE000243E579F022E578B41614E579C39472AA
:1071CE00500D9002417402F0900243E579F022E5F1
:1071DE0078D394004028E578C394155021E579D3EF
:1071EE009400401AE579C394FB5013900241740346
:1071FE00F0900242E578F0900243E579F022900299
:10720E000AE0FFEF64027065900211E0FEA3E0FF5A
:10721E00EF64014E702990021AE0FFEF70F89002B1
:10722E001DE4F0A3747FF0900215E0FEA3E0FF9042
:10723E00021FEEF0A3EFF09002197404F0D26290E8
:10724E000211E0FEA3E0FFEF64024E702090021ADE
:10725E00E0FFEF70F8900215E0FEA3E0FF90021D34
:0D726E00EEF0A3EFF09002197405F0D2626B
:01727B0022F0
:10FC0000C2AF12FCD812FD10E4F551F552E42552B2
:10FC1000FFE5513480FE12FCB6AD07AF52AE511273
:10FC2000FC5F0552E55270020551C3E551948040D6
:10FC3000DC755180755200AF52AE5112FCC7AD0752
:10FC4000AF52AE5112FC8A0552E55270020551C303
:10FC5000E55194F440E1D2AF75840075EF0122C202
:10FC6000AF75840F53A1FEE4F5B1F58443B701F5F8
:10FC700084438F018E088F098F828E83EDF0E4F527
:10FC800084538FFEF58453B7FE22C2AF75840F53A1
:10FC9000A1FE75B110E4F58443B701F584438F01EB
:10FCA0008E088F098F828E83EDF0E4F584538FFEEA
:10FCB000F58453B7FE22C2AF75B1218E0A8F0B8F28
:10FCC000828E83E493FF22C2AF75B1318E0A8F0B0F
:10FCD0008F828E83E493FF22C2AFE4FFFEE4F5B18E
:10FCE000F58443B701F584758F03AD07AC068C0826
:10FCF0008D098D828C83F0F58FF58453B7FE2FFF2D
:10FD000074043EFEC3948040D4E4F58453B7FE22CD
:10FD1000C2AF7F007E8075B110E4F58443B701F572
:04FD200084758F0354
:10FD2400AD07AC068C088D098D828C83F0F58FF5B8
:10FD34008453B7FE2FFF74043EFEC3648094744062
:08FD4400D1E4F58453B7FE225F
:101BC300C0D0C000C001C083C082C0E0C0F0C00765
:101BD300A291305001B37827E233F208E233F208DE
:101BE300E233F208E233F208E233F208E233F208B6
:101BF300E233F208E233F208E233F208E233F208A6
:101C0300E233F208E233F208E233F208E233F20895
:101C1300E233F208E233F208E233F208E233F20885
:101C2300E233F208E233F208E233F208E233F20875
:101C3300E233F208E233F208E233F208E233F20865
:101C4300E233F208E233F208E233F208E233F20855
:101C5300E233F208E233F208E233F208E233F20845
:011C6300E29E
:101C640033F208E233F208E233F208E233F208E234
:101C740033F208E233F2305D3A90214A784EE218AA
:101C8400203C03936028E218937023E21893601EAB
:101C9400E218937019E218936014E21893600FE24B
:101CA4001893700AE218937005E218936011C24BFE
:101CB400204C07C24BC24C021F23C24C021EF99097
:101CC400279A784E7F00E218203C03932FFFE218F6
:101CD400932FFFE218932FFFE218932FFFE218933C
:101CE4002FFFE218932FFFE218932FFFE218932F90
:101CF400FFE218932FFF90214A754100E2189313D5
:101D040092475003754138752200E21893139214D8
:101D1400500363411CE21893139213500363410E62
:0C1D2400E218931392125003634146E250
:101D300018931392115003634123E21893139210E6
:101D40008522425003634151752200E21893139299
:101D5000145003634168E2189313921350036341D4
:101D600075E21893139212500363417AE2189313A9
:101D70009211500363413DE2189313921085224360
:101D8000500363411F752200E2189313921750030A
:101D900063414FE218931392165003634126E218F1
:101DA000931392155003634152E218931392145007
:101DB00003634129E218931392135003634115E220
:101DC0001893139212500363410BE218931392116C
:101DD0005003634145E21893139210852244500347
:101DE000634162E218931392145003634131E21885
:101DF000931392135003634119E2189313921250F4
:101E00000363410DE218931392115003634107E2FB
:101E100018931392108522455003634143752200A5
:041E2000E21893131E
:101E24009216E21893139215E21893139214E2187F
:101E340093139213E21893139212E21893139211CC
:101E4400E21893139210852246E54665417025A257
:101E5400479248E54290004FF0E543900050F0E58A
:101E640044900051F0E545900052F0D24AC24BC272
:101E74004C021F2323F890269B93F990269AE8930B
:101E8400602EB40104B2478027B40205E8624280A0
:101E94001FB40305E862438017B40405E862448074
:101EA4000FB40505E862458007C24B304C7180458C
:101EB400204B04D24B801B204C0DD24C900058E098
:101EC400B50700400D8058900058E0B50700400267
:101ED4008023900058EFF0A247925A900054E542B4
:101EE400F0900055E543F0900056E544F09000571B
:101EF400E545F0802AA25A9248900054E090004FA1
:101F0400F0900055E0900050F0900056E0900051A1
:101F1400F0900057E0900052F0D24AC24BC24C12EB
:101F24001F37D007D0F0D0E0D082D083D001D000CA
:071F3400D0D022C0D0C00094
:101F3B00C0E0303F4EE553B40833A242B392B378BE
:101F4B007DE66036167882E6A2E7304401B3924212
:101F5B0092B2A2E7787EE633F6787FE633F67880A6
:101F6B00E633F67881E633F67882E633F6D553031B
:101F7B00755308D0E0D000D0D022C258D0E0D000AA
:101F8B00D0D022D0E0D000D0D022C0D0C000C00131
:101F9B00C083C082C0E0C0F0A291204F01B3780F84
:101FAB00E213F208E213F208E213F208E213F2086A
:101FBB00E213F208E213F208E213F208E213F2085A
:101FCB00E213F208E213F208E213F208E213F2084A
:101FDB00E213F208E213F208E213F208E213F2083A
:101FEB00E213F208E213F208E213F208E213F2082A
:051FFB00E213F208E210
:1020000013F208E213F290214A780FE20893139238
:102010000FE2089313920EE2089313920DE20893D5
:1020200013920CE2089313920BE2089313920AE2C4
:102030000893139209E20893139208852147E20856
:102040009313920FE2089313920EE2089313920DEA
:10205000E2089313920CE2089313920BE208931395
:10206000920AE20893139209E208931392088521D9
:1020700048E2089313920FE2089313920EE208933A
:1020800013920DE2089313920CE2089313920BE261
:10209000089313920AE20893139209C20885214912
:1020A000305D3DE54790249A854821300E02058336
:1020B00093602D14F875F003A490234B2582F582CC
:0B20C000E5F03583F583E493F9A3E419
:1020CB009390224A654993C965489329B4010050FE
:1020DB00048835D2411220F2D0F0D0E0D082D083E8
:1020EB00D001D000D0D022303D27C392B2788316D6
:1020FB00E6701E76087886E6A2E1304501B392B30E
:10210B00A2E17884E613F67885E613F67886E61373
:10211B00F622EF90234A75F003A42582F582E5831E
:10212B0035F0F583C23D7400937884F6740193788F
:10213B0085F67402937886F6C23FC23ED23D2200EA
:10214B000000000000000000000000000000000084
:10215B000000000000000000000000000001010072
:10216B000000000000000000000000000000010063
:10217B00000000000000010000000101010101004E
:10218B000000000000000000000000000000010043
:10219B000000000000000000000000000101010031
:1021AB000000000000000100000001000001010020
:1021BB000000010001010101010101010101010008
:1021CB000000000000000000000000000000010003
:1021DB0000000000000001000000010001010100EF
:1021EB0000000000000001000000010001010100DF
:1021FB0000000100010101000101010101010100C9
:10220B0000000000000001000000010001010100BE
:10221B0000000100010101000101010101010100A8
:10222B000000010001010100010101010101010098
:10223B000000010101010101010101010101010086
:10224B000101020102020301020203020303040162
:10225B000202030203030402030303030304050145
:10226B000202030203030402030304030404050232
:10227B000303040304040503040404040505060115
:10228B000202030203030402030303030404050213
:10229B0003030403030405030404050405050602F4
:1022AB0003030403040405030404050405050603E2
:1022BB0004040504050506040505060506060701C5
:1022CB0002020302030304020303040304040502D2
:1022DB0003030403040405030404050405050602B3
:1022EB0003030403040405030404050405050603A2
:1022FB000404050405050604050506050606070284
:10230B000303040304040503040405040505060381
:10231B000404050405050604050506050606070362
:10232B000404050405050604050506050606070451
:10233B00050506050606070506060706070708FD39
:10234B00D00C73700E3CF01AAF101E7F9022EC7005
:10235B0026D6F02ACBB02CA3F032BEB03417D03C2B
:10236B00B6D0461FB04E77F050F950526AB056DED9
:10237B009058BA306ACF3072D270745CD076E8F075
:10238B00786BD098E5709AF8309CBB50A40F70AA6C
:10239B007A70B26730B45DB0B8FCB0C26F50C6553E
:1023AB00D0CA3D90D489B0DA94F0DCD790E463B016
:1023BB00EA0BF0F43170F8DD310AB571148FF118B6
:1023CB00D1D126EB512AF6112C8B71463F5148B1D6
:1023DB00F14AACB14CC4F152D9B1546D915A2EF1B2
:1023EB0062BD116687916A9AD16CF29172D5517860
:1023FB0019F18C71B192D8D19A32D1AA47D1B25A74
:10240B0091B452F1C67531CC1D71D2A951DCD0B14A
:10241B00E85E11EA2B11F2EED212F392147D321612
:10242B00973226D8B232C5F234F7124AEA524C9F91
:0D243B005254A5D2582B725A7552644FD2DC
:1024480068C1726ADC326C78D2865F128C83729CA7
:102458004EB2A66972AC1C72B433D2CC18F2EABB85
:10246800330CCE33141EB32803F32EE51332F8537E
:102478003498735848F36472736845738617B39435
:102488007313A63C93B221D3B41B53B829B3C641E6
:10249800F3D8000000000000000000000000000069
:1024A8000000000000000000006A000000000000BA
:1024B800620D0000000000000000006F00480000EE
:1024C80000000000000000000000000000006C2276
:1024D80000000000000000000000000000000000F4
:1024E8005B00000000000000000000004100001E2A
:1024F8004759000000260000001D000010000035AC
:102508000000003D006B0043000000000000004B8D
:102518000005000000000000003800230000000053
:102528000000000000000000004C00000000000057
:102538000000000000000000000000000000320061
:1025480000040000000000000000000012600037D6
:102558000A00000000000000000000000008000061
:10256800611346000000000000254D340000572983
:1025780011000000000000640000000000000000DE
:10258800000000003A4A00002E4F190000001F000A
:1025980000000000006300000000000000270000A9
:1025A800001B000000000000000B5F3C006E5D4453
:1025B8000000006D00000000000000000053000053
:1025C800360000283F5E0000000000000000030005
:1025D8000030007000000069004067000000000043
:1025E8000055000042000021000000000000150016
:1025F80000000000000000000000005C0017000060
:102608000020000068020054000E58001C00000062
:1026180000000000005A000000000000002F000029
:10262800002B0000000024000000660039000000B4
:1026380000510000000900520000004500000000A1
:10264800000000310000002A0C000000001A000001
:10265800000000560000334E00000000000000009B
:102668000000002C1400003B07003E0000000000A2
:10267800000000000000001800001600502D0600A1
:1026880049000000000000000000650F0000000184
:102698000000000000000000060000000600060020
:1026A80005020600060006000404060005040208E8
:1026B80006000000060006000600060004080600E2
:1026C80006000600050806000600021006000600BF
:1026D800030100000600060002020600060004408E
:1026E80006000600041006000600060006000600A4
:1026F8000600060005100600060006000600060093
:102708000600010106000600060006000302060096
:102718000600000006000600050106000402020487
:102728000600060006000600060006000600060071
:1027380004800600020104200600060006000600C8
:102748000600060006000600060006000600060051
:102758000600060006000401060006000600060042
:102768000600031006000600060006000600060024
:10277800060006000600060006000600030806001C
:102788000600060006000304060006000600060010
:1027980006000002020402040406020404060406F9
:1027A80006080204040604060608040606080608C5
:0D27B80008060204040604060608040606CE
:1027C5000806080806040606080608080606080896
:1027D500060806060402040406040606080406069E
:1027E5000806080806040606080608080606080876
:1027F500060806060404060608060808060608086C
:10280500060806060406080806080606040806065D
:102815000406040402020404060406060804060667
:102825000806080806040606080608080606080835
:10283500060806060404060608060808060608082B
:10284500060806060406080806080606040806061D
:102855000406040402040606080608080606080815
:1028650006080606040608080608060604080606FD
:1028750004060404020608080608060604080606F7
:1028850004060404020806060406040402060404F9
:05289500020402020133
:030000000296194C
:0C961900787FE4F6D8FD7581A202602A7B
:10818C00BB010689828A83E0225002E722BBFE02F1
:09819C00E32289828A83E4932224
:1081A500BB010CE58229F582E5833AF583E022508F
:1081B50006E92582F8E622BBFE06E92582F8E222D9
:0D81C500E58229F582E5833AF583E49322F3
:1081D200BB010689828A83F0225002F722BBFE018C
:0281E200F32286
:1081E400EF8DF0A4A8F0CF8CF0A428CE8DF0A42EAF
:0281F400FE2269
:1081F600A3F8E0C5F025F0F0E5821582700215833C
:06820600E0C838F0E82298
:10820C00D083D082F8E4937012740193700DA3A301
:10821C0093F8740193F5828883E473740293686015
:06822C00EFA3A3A380DF15
:00000001FF
